:0200000480007A
:10000000B72F0000938F0F8073900F306F00400365
:100010001300000013000000130000001300000094
:100020001300000013000000130000001300000084
:100030001300000013000000130000001300000074
:100040009702000093824211739052309300000097
:10005000130100009301000013020000930200004E
:100060001303000093030000130400009304000036
:10007000130500009305000013060000930600001E
:100080001307000093070000130800009308000006
:100090001309000093090000130A0000930A0000EE
:1000A000130B0000930B0000130C0000930C0000D6
:1000B000130D0000930D0000130E0000930E0000BE
:1000C000130F0000930F000097110200938181C36A
:1000D00017050200130505479795030093850571E1
:1000E00013060000EF00001A17050200130545383B
:1000F000970502009385C54013060000EF008018A5
:1001000017A503001305C56E97B503009385056E0B
:1001100037B6ABAB1306B6BAEF00C01617B1030083
:100120001301016DEF8090369392120093D212006A
:100130009382D2FF638A02008322010013014100EF
:100140006F0000177300203083220100130141006B
:10015000730020301301C1FF23205100F32220340B
:10016000E3C402FC8322010013014100130141F8A2
:1001700023221100232421002326310023284100BB
:10018000232A5100232C6100232E71002320810299
:10019000232291022324A1022326B1022328C10293
:1001A000232AD102232CE102232EF1022320010570
:1001B0002322110523242105232631052328410567
:1001C000232A5105232C6105232E71052320810745
:1001D000232291072324A1072326B1072328C1073F
:1001E000232AD107232CE107232EF107732520347E
:1001F000F3251034130601006F000000731015344E
:1002000083204100032181008321C10003220101D9
:1002100083224101032381018323C10103240102BD
:1002200083244102032581028325C10203260103A1
:1002300083264103032781038327C1030328010485
:1002400083284104032981048329C104032A010569
:10025000832A4105032B8105832BC105032C01064D
:10026000832C4106032D8106832DC106032E010731
:10027000832E4107032F8107832FC1071301C10775
:10028000730020302320C5006376B50013054500B8
:100290006FF05FFF678000000000000000000000BA
:1002A000000000000000000000000000000000004E
:1002B000130101F8232011002322210023243100FF
:1002C0002326410023285100232A6100232C71009A
:1002D000232E8100232091022322A1022324B10294
:1002E0002326C1022328D102232AE102232CF10272
:1002F000232E010323201105232221052324310568
:100300002326410523285105232A6105232C710545
:10031000232E8105232091072322A1072324B1073F
:100320002326C1072328D107232AE107232CF1071D
:100330009702020083A2021723A02200F3221034A6
:10034000232E5106EF00C03B170102000321811547
:10035000032101008322C10773901234B7220000E9
:100360009382028873A00230832001000322C1001F
:100370008322010103234101832381010324C1015D
:100380008324010203254102832581020326C10241
:100390008326010303274103832781030328C10325
:1003A000832801040329410483298104032AC10409
:1003B000832A0105032B4105832B8105032CC105ED
:1003C000832C0106032D4106832D8106032EC106D1
:1003D000832E0107032F4107832F81071301010893
:1003E00073002030970202009382C21523A01200EE
:1003F00023A2220023A4320023A6420023A85200F5
:1004000023AA620023AC720023AE820023A09202D2
:1004100023A2A20223A4B20223A6C20223A8D202CC
:1004200023AAE20223ACF20223AE020323A01205A8
:1004300023A2220523A4320523A6420523A85205A0
:1004400023AA620523AC720523AE820523A092077E
:1004500023A2A20723A4B20723A6C20723A8D20778
:1004600023AAE20723ACF207EF60907017010200A5
:1004700003214103032101008322C1077390123439
:10048000B72200009382028873A00230832001000B
:100490000322C1008322010103234101832381013F
:1004A0000324C10183240102032541028325810223
:1004B0000326C10283260103032741038327810307
:1004C0000328C103832801040329410483298104EB
:1004D000032AC104832A0105032B4105832B8105CF
:1004E000032CC105832C0106032D4106832D8106B3
:1004F000032EC106832E0107032F4107832F810797
:1005000013010108730020309702020093828203D6
:1005100083A0020003A1420083A1820003A2C200C3
:1005200083A2020103A3420183A3820103A4C201A7
:1005300083A4020203A5420283A5820203A6C2028B
:1005400083A6020303A7420383A7820303A8C2036F
:1005500083A8020403A9420483A9820403AAC20453
:1005600083AA020503AB420583AB820503ACC20537
:1005700083AC020603AD420683AD820603AEC2061B
:1005800083AE020703AFC20983AF82076780000012
:1005900073700430130101F823201100232221007D
:1005A000232431002326410023285100232A6100FF
:1005B000232C7100232E8100232091022322A102EB
:1005C0002324B1022326C1022328D102232AE102D7
:1005D000232CF102232E01032320110523222105C0
:1005E000232431052326410523285105232A6105AB
:1005F000232C7105232E8105232091072322A10797
:100600002324B1072326C1072328D107232AE10782
:10061000232CF1079702020083A2C2E823A0220044
:10062000232E1106EF30007217010200032181E72B
:10063000032101008322C10773901234B722000006
:100640009382028873A00230832001000322C1003C
:100650008322010103234101832381010324C1017A
:100660008324010203254102832581020326C1025E
:100670008326010303274103832781030328C10342
:10068000832801040329410483298104032AC10426
:10069000832A0105032B4105832B8105032CC1050A
:1006A000832C0106032D4106832D8106032EC106EE
:1006B000832E0107032F4107832F810713010108B0
:1006C00073002030737004306F00000073104530E9
:1006D000678000007325403073F04330678000006E
:1006E00097070000938747FE232EB5FE2322C5FA05
:1006F000232635F82320F5F8130505F86780000058
:10070000130101FF23261100EF605043EF20501A20
:10071000631805008320C1001301010167800000F8
:100720008320C100130101016F30C0619307850070
:100730001307F0FF2322F5002324E5002326F5000C
:100740002328F500232005006780000023280500EA
:10075000678000008327450023A2F50003A78700D8
:1007600023A4E50003A787002322B70023A4B70032
:1007700023A8A50083270500938717002320F500F1
:100780006780000003A605009307F0FF13078500AC
:100790006316F6006F008003138707008327470066
:1007A00083A60700E37AD6FE23A2F50023A4B700B0
:1007B00023A4E5002322B70023A8A5008327050072
:1007C000938717002320F5006780000003270501A9
:1007D000832747006FF05FFD0327450083268500D0
:1007E000832705012324D70003278500832645009E
:1007F0002322D70003A747006316A700032785001D
:1008000023A2E7002328050003A507001305F5FF31
:1008100023A0A70067800000130101FF23248100AB
:1008200023261100232291008327050413040500C9
:100830006398070283270500638C070C13050000EB
:100840008327840393871700232CF4028320C1009D
:10085000032481008324410013010101678000000B
:1008600093040600631A0604032585001386070017
:10087000EF501009832784008326040403274400D3
:10088000B387D7002324F400E3EAE7FA83270400C0
:10089000130500002324F4008327840393871700A3
:1008A000232CF4028320C10003248100832441000F
:1008B00013010101678000000325C50013860700AE
:1008C000EF501004032704048327C4008326040088
:1008D0003307E040B387E7002326F40063F8D7002E
:1008E000832744003387E7002326E4009307200092
:1008F000E396F4F483278403E38207F483278403D5
:10090000130500009387F7FF232CF4026FF05FF3C9
:1009100003254500EF305069232204006FF05FF299
:10092000130101FE232E1100232C8100232A9100A4
:10093000032445052326A100630E04020327840334
:100940008327C4036366F700737004306F000000F0
:1009500003278403930400006362F7028320C1012C
:100960000324810113850400832441011301010242
:1009700067800000737004306F000000138605006C
:10098000130504009305C100EFF01FE90327840459
:100990009307F0FF93040500630AF700832784049C
:1009A000938717002324F4046FF05FFB832744022E
:1009B000E38607FA13054402EF30101BE30005FA43
:1009C000930410006FF09FF9032605049387050038
:1009D000630406028325C50003274500B385C500CF
:1009E0002326B50063E6E500832505002326B50030
:1009F000138507006F50C07067800000130101FD70
:100A000023248102232611021304050023229102CC
:100A100023202103232E3101232C4101232A5101BC
:100A2000EF30906583278404635CF004130A44026A
:100A30009309F0FF1309100083244405638E04001A
:100A400003A7840383A7C403232681006368F70AEE
:100A5000737004306F000000832744026382070232
:100A600013050A00EF3050106314050C832784042B
:100A70009387F7FF2324F40483278404E34EF0FADA
:100A80009307F0FF2324F404EF305062EF30D05E80
:100A900083274404635CF002832704016388070210
:100AA0009304040113850400EF30100C631605084D
:100AB000832744049387F7FF2322F4048327440405
:100AC0006356F00083270401E39E07FC9307F0FFC1
:100AD0002322F404EF30905D8320C10203248102BD
:100AE00083244102032901028329C101032A8101D0
:100AF000832A4101130101036780000003A78403D7
:100B0000E376F7F6130600009305C1001385040091
:100B1000EFF09FD083A78404930A05006382370314
:100B200083A784049387170023A4F404E3902AF591
:100B3000EF30D0306FF09FF3EF3050306FF05FF751
:100B400083A74402E38407FE13854402EF30D001FB
:100B5000E30E05FC6FF0DFFD63000508130101FFE4
:100B60002324810023229100130405002326110071
:100B700093840500EF305050832604048327C40378
:100B800003270400232C0402B387F6021306F0FFA8
:100B90002322C4042324E4002324C404B386D740BE
:100BA000B307F7003307D7002322F4002326E4001D
:100BB0006398040283270401639E0702EF30104FFD
:100BC0008320C10003248100832441001305100009
:100BD0001301010167800000737004306F00000092
:100BE00013050401EFF09FB413054402EFF01FB4A6
:100BF0006FF0DFFC13050401EF300077930710005E
:100C0000E31EF5FAEFF0DF986FF05FFB6316050067
:100C1000737004306F000000130101FE232A91005D
:100C20002328210123263101232E1100232C8100AA
:100C30009309060013890500930405006380050AE3
:100C40003305B50213059505EF50002B130405007D
:100C5000630E0508930785052320F500232E9402D3
:100C600023202405EF305041832604048327C40346
:100C7000032704001306F0FFB387F602232C0402B7
:100C80002322C4042324E4002324C4041305040100
:100C9000B386D740B307F7003307D7002322F40009
:100CA0002326E400EFF09FA813054402EFF01FA8ED
:100CB000EF30D03F23083405232A04041305040031
:100CC0008320C101032481018324410103290101FF
:100CD0008329C1001301010267800000130580050C
:100CE000EF50802113040500631605007370043073
:100CF0006F000000232084006FF05FF6130101FDF8
:100D00002322910293040500130580052324810208
:100D10002326110223202103232E3101232C4101FC
:100D2000EF50801D1304050063080506232C0502FF
:100D30009307F0FF2322F50413071000130A05019F
:100D40002324F40413050A00232EE40223220400C2
:100D50002320040023240400232604002320040469
:100D600023089404232A0404EFF05F9C130944022F
:100D700013050900EFF09F9B832704042322010041
:100D8000638E0702737004306F00000013050400C7
:100D9000EFF0DFC6EF204057130504008320C102A7
:100DA0000324810283244102032901028329C10112
:100DB000032A81011301010367800000EF30100C4A
:100DC000631605008327410063980710EF30D02A8F
:100DD000032784038327C403930400009309F0FFCF
:100DE0006362F70883274100638E070A6396040055
:100DF00013058100EF300072EF30502BEF20401DC3
:100E0000EF3090278327440463943701232204049E
:100E1000832784046394370123240404EF301029CA
:100E20009305410013058100EF30C071E31005F612
:100E3000EF309024032784038327C4036308F70655
:100E4000EF30D02613050400EFF05FBBEF20C04B5E
:100E500093041000EF305022032784038327C40338
:100E6000E372F7F803260404631C060683270400D4
:100E7000638A070A130500008327840303274405B8
:100E800093871700232CF4026306070893050000DC
:100E900013050400EFF0DFA8930710006314F500BA
:100EA000EFF00FEFEF3090206FF01FEFEF301020DA
:100EB0008325410013050A00EF30001E13050400CE
:100EC000EFF0DFB3EF204044E31405F8EFF04FEC10
:100ED000930410006FF01FF8737004306F0000006F
:100EE0000325840093050000EF50802183278400B0
:100EF0008326040403274400B387D7002324F40087
:100F0000E3EAE7F683270400130500002324F40036
:100F10006FF09FF683274402639E0700E30405F801
:100F20006FF01FF803254400EF301008232204005F
:100F30006FF09FF413050900EF3000439307100092
:100F4000E312F5F66FF0DFF56316050073700430F9
:100F50006F0000006376B500737004306F0000000E
:100F6000130101FF232481001306200013840500D0
:100F70009305000023261100EFF05FC9630C050004
:100F8000232C85028320C100032481001301010169
:100F900067800000737004306F000000130101FCD3
:100FA000232E1102232C8102232A910223282103BC
:100FB00023263103232441032322510323206103E9
:100FC0002326C10063040516638A051493072000D5
:100FD000639CF6000327C503930710006306F70020
:100FE000737004306F0000009384060013890500BD
:100FF00013040500EF308068631A05008327C100E1
:1010000063860700737004306F000000EF30D00675
:10101000032784038327C40393090000130B2000D4
:10102000130AF0FF930A04016364F70863846411F0
:101030008327C100638C071C639609001305810197
:10104000EF30404DEF309006EF109078EF30D00247
:1010500083274404639447012322040483278404E0
:101060006394470123240404EF3050049305C10026
:1010700013058101EF30004D63100518EF30C07F7C
:10108000032784038327C4036304F706EF301002A9
:1010900013050400EFF09F96EF200027930910003E
:1010A000EF30807D032784038327C403E370F7F8C0
:1010B00003260404630406086390041603258400D1
:1010C00093050900EF50C00383278400832604049E
:1010D00003274400B387D7002324F40063E4E70622
:1010E00083270400130500002324F4006F00C005CB
:1010F000EF30C07B8325C10013850A00EF20D07933
:1011000013050400EFF09F8FEF200020E31805F88F
:10111000EFF00FC8930910006FF09FF883270504C4
:10112000E38607EA737004306F00000073700430C8
:101130006F000000032604046314060683270400DE
:10114000638C0710130500008327840303274405DD
:1011500093871700232CF4026306070E938504007F
:1011600013050400EFF0CFFB930710006302F50EA8
:10117000EF30C073130510008320C10303248103E3
:1011800083244103032901038329C102032A810225
:10119000832A4102032B010213010104678000002E
:1011A0000325C40093050900EF40907583270404CC
:1011B0000327C40083260400B307F0403307F70079
:1011C0002326E400637CD70003274400B307F7001D
:1011D0002326F40093072000E396F4F68327840384
:1011E000E38207F683278403130500009387F7FF44
:1011F000232CF4026FF05FF513050400EFF01F805D
:10120000EF208010130500006FF01FF7EF30006A29
:10121000130500006FF05FF60325C4009305090075
:10122000EF40106E832704040327C40083260400C4
:10123000B307F0403307F7002326E400E37CD7F838
:101240006FF09FF88327440263900702E30205F2E0
:10125000EFF00FB46FF0DFF103254400EF30C0541E
:10126000232204006FF05FEE13054402EF30C00F3D
:1012700093071000E31EF5EE6FF09FFD6304050475
:10128000130101FF23248100232291002326110052
:10129000232021010329450013040500EF30003D00
:1012A000930400006304A9028320C1000324810089
:1012B0001385040003290100832441001301010167
:1012C00067800000737004306F0000008327C40043
:1012D000930410009387F7FF2326F400E39607FC9E
:1012E0009306000013060000930500001305040098
:1012F000EFF0DFCA6FF05FFB6302050A6388050841
:10130000130101FE232C8100232A910023282101AF
:1013100023244101232E11002326310193072000AD
:101320009384060013090600138A050013040500C0
:10133000639CF6000327C503930710006302F70AB6
:10134000737004306F000000EFF0CFB80327840300
:101350008327C403930905006366F7049304000020
:1013600013850900EFF08FB68320C10103248101AA
:101370001385040003290101832441018329C1004D
:10138000032A8100130101026780000083270504FE
:10139000E38807F6737004306F0000007370043048
:1013A0006F00000003260404631E060C832704005C
:1013B00063880712832784031307F0FF93871700BE
:1013C000232CF402832784046388E70E8327840494
:1013D00093041000938717002324F4046FF05FF840
:1013E000EFF04FAF032784038327C403930905005D
:1013F0006360F70603260404E30A06FA0325C40023
:1014000093050A00EF40D04F832704040327C4004C
:1014100083260400B307F0403307F7002326E400D7
:101420006378D70003274400B307F7002326F400AE
:1014300093072000E390F4F883278403E38C07F6F6
:10144000832784039387F7FF232CF4026FF09FF622
:1014500003260404E30C06F40325C40093050A00E4
:10146000EF40104A832704040327C40083260400A6
:10147000B307F0403307F7002326E400E364D7FA0C
:101480006FF09FFBE39C04F60325840093050A009C
:10149000EF40104783278400832604040327440079
:1014A000B387D7002324F400E3E6E7F083270400A2
:1014B0002324F4006FF01FF083274405638A07029A
:1014C0009385040013050400EFF08FC5930410000A
:1014D000E31895E8E30609E8232099006FF05FE838
:1014E00003254400EF30402C232204006FF09FECD2
:1014F0008327440293041000E38407E613054402A3
:10150000EF209066E31805FC6FF09FE56302050A83
:101510008327050463860700737004306F000000A2
:1015200083270500638A0708130101FE232C81002D
:10153000232A9100130405002328210123263101C9
:10154000232E110013890500EFF0CF9803278403A1
:101550008327C40393090500930400006376F70210
:10156000832784031307F0FF93871700232CF402CB
:1015700083278404638AE704832784049304100088
:10158000938717002324F40413850900EFF00F94C8
:101590008320C10103248101138504000329010173
:1015A000832441018329C1001301010267800000E7
:1015B000737004306F00000083274500E38607F650
:1015C000737004306F0000008327440563800702B6
:1015D0009305000013050400EFF08FB4930710008B
:1015E0006300F502930410006FF01FFA8327440292
:1015F000E38A07FE13054402EF201057E30405FEBB
:10160000E30209FE930710002320F9006FF09FFD0D
:10161000130101FC232E1102232C8102232A9102A3
:101620002328210323263103232441032326C10039
:101630006300051663860514938906001389050067
:1016400013040500EF308003631A05008327C100EF
:1016500063860700737004306F000000EF30C02114
:1016600083278403639E070A8327C10063880718C2
:1016700013058101EF20106A9304F0FF130A44025E
:101680006F008002EF30802213050400EFF00FB7E7
:10169000EF109047EF30401E8327840363920708C2
:1016A0008327C100638C0714EF304020EF105012E5
:1016B000EF30801C832744046394970023220404A2
:1016C000832784046394970023240404EF30001ECE
:1016D0009305C10013058101EF20D0666316051044
:1016E000EF30801983278403E39E07F8EF30001C56
:1016F000832704006386070A8325C10013050A00B7
:10170000EF20901913050400EFF04FAFEF10D03F1A
:1017100063040508EF30401683278403E38207F84B
:1017200093050900130504008324C400EFF0CFA93A
:101730006392090883278403032704009387F7FF34
:10174000232CF40263160700EF30801D2322A4002F
:101750008327040163900708EF304015130510003C
:101760008320C1030324810383244103032901034C
:101770008329C102032A810213010104678000004A
:1017800083270504E38A07EA737004306F000000C2
:10179000737004306F000000EFE09FDF6FF09FF781
:1017A000EF30800D03254400EF201070EF30001063
:1017B0006FF09FF48327440223269400E38E07F8FA
:1017C00013054402EF20503AE30805F8EFE05FDC30
:1017D0006FF09FF813050401EF20103993071000F4
:1017E000E31CF5F66FF09FFE13050400EFF00FA168
:1017F000EF109031130500006FF09FF6EF30000BF3
:10180000130500006FF0DFF563000506130101FF0B
:10181000232481002320210123261100232291006B
:10182000832445001389050013040500EF2010648C
:101830006380A404930600001306090093050000CA
:1018400013050400EFF0DFDC93071000630CF502D2
:101850008320C10003248100832441000329010067
:101860001301010167800000737004306F000000F5
:101870008327C40013051000938717002326F40064
:101880006FF01FFD8327C400938717002326F40001
:101890006FF01FFC630805066386050C130101FE4B
:1018A000232C8100232A91002328210123263101A2
:1018B0002324410113040500232E110013090600FF
:1018C00093890500EFE01FE183278403130A0500D5
:1018D00093040000639C070213050A00EFE01FDF7A
:1018E0008320C10103248101138504000329010120
:1018F000832441018329C100032A810013010102CD
:1019000067800000737004306F0000000326040439
:10191000630406028325C40083274400B385C50001
:101920002326B40063E6F500832504002326B400D3
:1019300013850900EF40C07C832784031307F0FF61
:101940009387F7FF232CF402832744046384E70280
:101950008327440493041000938717002322F40480
:101960006FF09FF783270504E38A07F27370043052
:101970006F000000832704016396070093041000A2
:101980006FF09FF513050401EF20101EE30805FE1C
:10199000E30609FE930710002320F9006FF01FFEF5
:1019A0006306050883270504638A0508638407081E
:1019B000130101FE232C8100232A910023282101F9
:1019C0002324410113040500232E11002326310195
:1019D000138A0500EFE01FD0832784031309050055
:1019E00093040000638E07008329C40093050A0056
:1019F00013050400EFE05FFD93041000232634017B
:101A000013050900EFE09FCC8320C101032481016D
:101A10001385040003290101832441018329C100A6
:101A2000032A8100130101026780000073700430F3
:101A30006F000000737004306F000000E38C07FE3D
:101A4000737004306F00000063160500737004307B
:101A50006F000000130101FF23248100130405001F
:101A600023261100EF20506103248403EF2010642B
:101A70008320C10013050400032481001301010128
:101A80006780000063160500737004306F0000006B
:101A9000130101FF232611002324810013040500F4
:101AA000EF20905D832784030324C4033304F440B0
:101AB000EF20D05F130504008320C10003248100C0
:101AC00013010101678000006306050003258503FB
:101AD00067800000737004306F0000006308050425
:101AE00097870300938747CC03A747006304E50467
:101AF00003A7C7006302E50803A74701630AE506D9
:101B000003A7C7016302E50603A74702630AE504CA
:101B100003A7C7026302E50403A74703630AE502BC
:101B200003A7C7036302E5026F40005573700430DA
:101B30006F0000001307000013173700B387E7009A
:101B400023A007006F404053130770006FF0DFFEC3
:101B5000130760006FF05FFE130750006FF0DFFDAA
:101B6000130740006FF05FFD130730006FF0DFFCDC
:101B7000130720006FF05FFC130710006FF0DFFB0E
:101B80000325C504678000002326B5046780000094
:101B900003450505678000006308050003258503EC
:101BA0001335150067800000737004306F0000006B
:101BB000630C0500832785030325C5033305F54022
:101BC0001335150067800000737004306F0000004B
:101BD00097870300938747BD03A7070063000704A7
:101BE00003A787006308070403A707016308070426
:101BF00003A787016308070403A707026308070414
:101C000003A787026308070403A70703630C0704FD
:101C100003A787036304070467800000130700001D
:101C200013173700B387E70023A0B70023A2A7004C
:101C300067800000130710006FF09FFE130720005D
:101C40006FF01FFE130730006FF09FFD1307400079
:101C50006FF01FFD130750006FF09FFC130770001B
:101C60006FF01FFC130760006FF09FFB9787030066
:101C7000938787B303A747006300E50403A7C70062
:101C80006306E50403A747016306E50403A7C7014C
:101C90006306E50403A747026306E50403A7C7023A
:101CA0006306E50403A74703630AE50403A7C70324
:101CB0006302A704678000001307000013173700B2
:101CC000B387E70023A00700678000001307100018
:101CD0006FF0DFFE130720006FF05FFE1307300088
:101CE0006FF0DFFD130740006FF05FFD130750003A
:101CF0006FF0DFFC130770006FF05FFC13076000EC
:101D00006FF0DFFB130101FD2324810223229102E6
:101D1000232021031304050023261102232E310161
:101D2000232C4101232A5101938405001309060045
:101D3000EF209034032744049307F0FF6314F70067
:101D400023220404032784049307F0FF6314F7009D
:101D500023240404EF20903583278403639A07002B
:101D6000130609009385040013054402EF20004F79
:101D7000EF20903083278404635CF004130A44024C
:101D80009309F0FF1309100083244405638E0400B7
:101D900003A7840383A7C403232681006368F70A8B
:101DA000737004306F0000008327440263820702CF
:101DB00013050A00EF20405B6314050C832784049D
:101DC0009387F7FF2324F40483278404E34EF0FA77
:101DD0009307F0FF2324F404EF20502DEF20D029A7
:101DE00083274404635CF0028327040163880702AD
:101DF0009304040113850400EF20005763160508BF
:101E0000832744049387F7FF2322F40483274404A1
:101E10006356F00083270401E39E07FC9307F0FF5D
:101E20002322F404EF2090288320C102032481029E
:101E300083244102032901028329C101032A81016C
:101E4000832A4101130101036780000003A7840373
:101E5000E376F7F6130600009305C100138504002E
:101E6000EFE09F9B83A78404930A050063823703F6
:101E700083A784049387170023A4F404E3902AF52E
:101E8000EF20C07B6FF09FF3EF20407B6FF05FF798
:101E900083A74402E38407FE13854402EF20C04C6D
:101EA000E30E05FC6FF0DFFD631605007370043070
:101EB0006F000000130101FF23229100930405002D
:101EC00013152500130595052324810023261100F1
:101ED000EF4080021304050063040508930785059D
:101EE0002320F50093074000232E95022320F504BC
:101EF000EF209018832604048327C40303270400DB
:101F00001306F0FFB387F602232C04022322C40435
:101F10002324E4002324C40413050401B386D7401A
:101F2000B307F7003307D7002322F4002326E40089
:101F3000EFE0CFFF13054402EFE04FFFEF20101753
:101F400023080404232A0404130504008320C10089
:101F500003248100832441001301010167800000F4
:101F6000737004306F000000130101FF232481000F
:101F700023229100232021011304050023261100B0
:101F800013890500EF20500F8327440593040000B8
:101F900063820702EF2090118320C1000324810097
:101FA000138504000329010083244100130101016A
:101FB000678000008327840393040000E39C07FCF0
:101FC000232A2405930410006FF0DFFC83274505C6
:101FD0006388B7009307000013850700678000003F
:101FE0000327850393070000E31807FE130101FF91
:101FF000232481001304050023261100EF20D007BD
:10200000232A0404EF20900A8320C10003248100C6
:10201000930710001385070013010101678000007A
:10202000130101FE13860500930600009305C1000D
:10203000232E110023260100EFF08FDD8320C10144
:102040000325C1001301010267800000130101FE96
:10205000232E1100232C8100232A91002326010026
:10206000630C050213040500EFE0CFE68327840329
:10207000930405006396070213850400EFE00FE563
:102080008320C101032481010325C1008324410170
:102090001301010267800000737004306F000000BC
:1020A00003260404630406028325C4008327440036
:1020B000B385C5002326B40063E6F500832504003C
:1020C0002326B4001305C100EF4080038327840357
:1020D0001307F0FF9387F7FF232CF40283274404B0
:1020E000638AE70083274404938717002322F404BC
:1020F0006FF09FF883270401E38007F813050401BC
:10210000EF2080266FF05FF763040504130101FDE3
:10211000232E3101232C410123261102138A0700AB
:10212000232481022322910223202103232A510107
:102130002328610123267101232481019307900044
:102140009309070063FAE700737004306F00000022
:10215000737004306F000000930A0500938405003B
:1021600013090600938B0600130B08006304082C68
:1021700013050006EF305058130405006304052AC8
:102180001319290023286503130609009305500A33
:1021900013050B00EF40C00803C7040083270403A6
:1021A0001309C9FF230AE40203C704003389270186
:1021B0001379C9FF6306070E83C71400A30AF4024C
:1021C00083C71400638E070C83C72400230BF4021B
:1021D00083C724006386070C83C73400A30BF40273
:1021E00083C73400638E070A83C74400230CF402BC
:1021F00083C744006386070A83C75400A30CF40214
:1022000083C75400638E070883C76400230DF4025C
:1022100083C764006386070883C77400A30DF402B4
:1022200083C77400638E070683C78400230EF402FD
:1022300083C784006386070683C79400A30EF40255
:1022400083C79400638E070483C7A400230FF4029E
:1022500083C7A4006386070483C7B400A30FF402F6
:1022600083C7B400638E070283C7C4002300F4044D
:1022700083C7C4006386070283C7D400A300F404A5
:1022800083C7D400638E070083C7E4002301F404EE
:1022900083C7E4006386070083C7F400A301F40446
:1022A000130B440013050B00A3010404232634037D
:1022B00023283405232A0404EFE04FC913058401C1
:1022C000EFE0CFC89307A000B3873741232C040465
:1022D00023288400232CF4002322840223220404D4
:1022E000232E040413860B0093850A0013050900AE
:1022F000EFE00FBF2320A40063040A0023208A001C
:102300007370043017E901001309091883270900C5
:1023100097E4010093840419638C070003A7040069
:1023200083A7040083274704938717002322F70419
:1023300017E7010013070716832707009387170085
:1023400097E6010023A8F61483A704006380071012
:102350008327090017EA0100130A8A26639C0700F5
:1023600083A7040083A7C70263E6F90097E701008B
:1023700023AA871297E701009387071003A7070096
:1023800097E60100938686108327C40283A6060081
:102390001307170017E601002320E60E2324E404A8
:1023A00063F6F60017E701002322F70E130740013A
:1023B000B387E70293050B003305FA00EFE08FB90E
:1023C000832709006388070083A7040083A74704C5
:1023D000639E07088327090013041000638A07001F
:1023E00083A7040083A7C70263F43701EFE04F9A85
:1023F000130504008320C1020324810283244102C7
:10240000032901028329C101032A8101832A410191
:10241000032B0101832BC100032C81001301010355
:102420006780000013050B00EF3010451304F0FF28
:102430006FF01FFC13152600EF30102C130B050056
:10244000E31805D21304F0FF6FF09FFA97E701003D
:1024500023AA87040327070093071000630AF702E3
:1024600017EA0100130ACA156FF0DFF003A7040092
:1024700083A60400832747049387F7FF2322F704EA
:1024800083A74604E39807F4736004306FF09FF469
:10249000930A000017EA0100130A8A12130C400184
:1024A000930BA00033858A03938A1A003305AA0090
:1024B000EFE0CFA7E3987AFF97EB0100938BCB1C5B
:1024C00013850B00EFE08FA697EA0100938A0A1D9F
:1024D00013850A00EFE08FA517E501001305451DE0
:1024E000EFE0CFA417E501001305C51DEFE00FA431
:1024F00017E501001305451EEFE04FA397E7010024
:1025000023A077FB97E7010023AA57F96FF09FE616
:10251000130101FF232481002326110023229100AF
:1025200023202101130405007370043097E4010097
:10253000938484F583A70400639E07106318040046
:1025400097E70100938707F603A4070013094400E7
:1025500013050900EFE04FA8832784026386070074
:1025600013058401EFE04FA79305090017E501006B
:1025700013054515EFE00F9E97E701009387C7F11C
:1025800003A7070097E70100938707EF83A70700DA
:102590001307170097E6010023A0E6F003A7040045
:1025A0009387170097E6010023A8F6EC630C070059
:1025B00097E70100938707EF03A707000327470466
:1025C000631C070E83A70400638A070697E70100D0
:1025D000938747ED03A707006302871073700430E9
:1025E00003A704006318070817E70100130747EB68
:1025F0008326070083A606006392060A1307F0FFEE
:1026000097E6010023A8E6E603A704006308070293
:1026100003A70700032747046302070203A7070075
:1026200083A60700832747049387F7FF2322F70435
:1026300083A7460463940700736004308320C100BD
:1026400003248100832441000329010013010101B7
:102650006780000097E701009387C7E403A707009E
:1026600083A7070083274704938717002322F704D3
:102670006FF0DFEC83A6070003A7070003A746045B
:102680001307170023A2E60417E70100130747E129
:102690008326070083A60600E38206F603270700C9
:1026A0000327C7000327C7000327470097E6010059
:1026B00023A2E6DC6FF05FF503A7070083A60700FF
:1026C000832747049387F7FF2322F70483A7460451
:1026D000E39A07EE736004306FF0DFEE97E70100D6
:1026E000938707D983A707006386070073700430B8
:1026F0006F000000032481008320C1008324410077
:1027000003290100130101016FD09FE86304050C48
:1027100017E70100130707D9832607009307000076
:102720006386A60A130101FF2326110023248100DA
:10273000232291007370043097E601009386C6D47B
:1027400083A70600638C0700032607008327070082
:1027500083274604938717002322F60483A70600E5
:1027600093040500032445016388070083270700BD
:1027700083A747046394070697E70100938747D22E
:1027800083A70700638C870697E70100938707D12B
:1027900083A707006384870697E701009387C7F341
:1027A0006306F40497E701009387C7F1630CF40212
:1027B000930710008320C10003248100832441007B
:1027C00013850700130101016780000013850700CE
:1027D00067800000737004306F000000EF60403BC2
:1027E0006FF09FF9930740006FF0DFFC83A784022E
:1027F00093B71700938727006FF0DFFB9307200044
:102800006FF05FFB7370043097E701009387C7C7D1
:1028100003A70700631607026304050483A70700E4
:102820000325C502638C070097E70100938787C7DC
:1028300003A7070003274704631C07026780000003
:1028400017E70100130707C68326070003270700C1
:1028500003A746041307170023A2E604E31005FCB0
:1028600017E70100130707C4032507006FF01FFBDC
:1028700003A7070083A60700832747049387F7FF72
:102880002322F70483A74604E39A07FA736004300F
:1028900067800000130101FF232481001304050059
:1028A00023261100EFD01FE36318040097E701000F
:1028B000938747BF03A407000324C402EFD01FE19E
:1028C0008320C100130504000324810013010101CA
:1028D000678000009307900063F6B70073700430C0
:1028E0006F000000130101FE232C8100232E110034
:1028F000232A910023282101232631012324410189
:10290000130405007370043017E901001309C9B7F7
:1029100083270900639207106300041283270405CC
:10292000638EF50A17E701001307C7B763F0B70214
:1029300083260700638E8612032707008324C702BD
:10294000B3B4950093C414006F0000018324070002
:10295000B384844093B414000327C4026386E70E53
:10296000832784012328B40463C807009307A000C9
:10297000B385B740232CB40093172700B387E70033
:102980000327440197E90100938989C3939727009E
:10299000B387F9006310F704130A440013050A0013
:1029A000EFD09FE317E70100130747AE8327C40268
:1029B000032707006376F70017E701002328F7AC29
:1029C00013074001B387E70293050A003385F90036
:1029D000EFD05FD863840400EFD09FBB832709004A
:1029E000638C070097E701009387C7AB83A70700B5
:1029F00083A74704639E07048320C1010324810148
:102A000083244101032901018329C100032A810094
:102A1000130101026780000097E70100938787A8F0
:102A200003A7070083A7070083274704938717009E
:102A30002322F704E31404EE97E70100938787A6A7
:102A400003A407006FF09FED2326B4026FF05FF13F
:102A5000032481018320C101832441010329010151
:102A60008329C100032A8100130101026F60401213
:102A7000930400006FF05FEE630A0508130101FE86
:102A8000232A910097E401009384C4A183A7040042
:102A9000232E1100232C810023282101232631011C
:102AA0006388A7047370043017E901001309C99DF6
:102AB00083270900638C070003A7040083A7040091
:102AC00083274704938717002322F7040327450130
:102AD00097E70100938747C0630EF7028327090039
:102AE0006388070083A7040083A74704639E070841
:102AF0008320C101032481018324410103290101B1
:102B00008329C10013010102678000007370043043
:102B10006F0000008327850217E70100130747B9FC
:102B2000E38EE7FAE39C07FA9309450013040500D6
:102B300013850900EFD05FCA17E701001307079557
:102B40008327C402032707006376F70017E7010015
:102B5000232EF79213074001B387E70217E5010020
:102B6000130505A6938509003305F500EFD09FBE38
:102B700083A704000327C40283A7C702E360F7F614
:102B8000EFD01FA16FF09FF5032481018320C101C5
:102B900083244101032901018329C100130101029A
:102BA0006F50107F63020506130101FE232C810084
:102BB000232A91002328210113040500232E11004C
:102BC00023263101EFD01FB10327440197E701000D
:102BD000938787B01309050093040000630AF70286
:102BE00013050900EFD09FAE8320C10103248101AA
:102BF0001385040003290101832441018329C100B5
:102C00001301010267800000737004306F00000040
:102C10008327840217E50100130585A9E382A7FC39
:102C2000E39007FC97E701009387878483A7070059
:102C30006394070697E701009387C78683A7070079
:102C40008324C4029309440083A7C70213850900A3
:102C5000B3B4F400EFD05FB817E7010013070783A0
:102C60008327C4020327070093C414006376F70088
:102C700017E70100232CF78013074001B387E70211
:102C800017E501001305C593938509003305F50089
:102C9000EFD05FAC6FF0DFF493058401EFD09FAB12
:102CA0006FF01FF4130101FE37150000232E1100F1
:102CB000232C8100232A910023282101232631017E
:102CC000232441012322510123206101EF30C0223E
:102CD000630805229304050013050006EF30C021A8
:102CE0001304050063040526371600009305500AF7
:102CF0002328950213850400EF30805283240403B7
:102D0000B71700009387C7FFB384F400B7474C455B
:102D100093879744130A4400232AF40213050A00F8
:102D2000230C0402A3010404232604022328040420
:102D3000232A0404EFD09FA113058401EFD01FA123
:102D40009307A000232C040493F4C4FF23288400D9
:102D5000232CF4002322840223220404232E0404BF
:102D600013060000971500009385C5EA138504003B
:102D7000EFD01F972320A4007370043017D90100EF
:102D8000130989708327090097D401009384847103
:102D9000638C070003A7040083A70400832747046C
:102DA000938717002322F70417D701001307876EB4
:102DB000832707009387170097D6010023ACF66C92
:102DC00083A704006388070A8327090097D90100B5
:102DD0009389097F639C070083A7040083A7C70228
:102DE0006396070097D7010023AE876A97D7010043
:102DF0009387876803A7070097D601009386066923
:102E00008327C40283A606001307170017D6010004
:102E10002324E6662324E40463F6F60017D70100B2
:102E20002326F766139527003305F50013152500B3
:102E300093050A003385A900EFD0DF9183270900AD
:102E40006388070083A7040083A74704639E070CD9
:102E5000832709006384070083A70400EF2050063E
:102E600093071000630AF510631C050873700430A3
:102E70006F00000097D7010023A687620327070091
:102E80009307100097D9010093898973E310F7F62F
:102E9000938A090017DB0100130B0B7F13850A00CF
:102EA000938A4A01EFD09F88E31A5BFF17D5010090
:102EB0001305857DEFD09F8797DA0100938A0A7EFC
:102EC00013850A00EFD09F8617D501001305457EB4
:102ED000EFD0DF8517D501001305C57EEFD01F8524
:102EE00017D501001305457FEFD05F8497D7010008
:102EF00023A8675B97D7010023A2575B6FF01FEFF2
:102F00008320C1010324810183244101032901019C
:102F10008329C100032A8100832A4100032B010079
:102F2000130101026780000003A7040083A60400C8
:102F3000832747049387F7FF2322F70483A74604D8
:102F4000E39807F0736004306FF09FF00324810171
:102F50008320C101032901018329C100032A8100C3
:102F6000832A4100032B01001385040083244101BF
:102F7000130101026F304010737004309307F0FFAB
:102F800017D701002328F74E0324810197D70100AA
:102F900023ACA74E8320C1018324410103290101F1
:102FA0008329C100032A8100832A4100032B0100E9
:102FB00097D7010023AE074C130101026FD08FC2D7
:102FC0007370043097D7010023A0074C6FD0CFD384
:102FD00017D701001307C7498327070093871700F6
:102FE0002320F700678000007370043097D701003A
:102FF0009387874903A707006318070217D70100C3
:10300000130707490325070083A70700638C070000
:1030100097D701009387074903A7070003274704B1
:10302000631407026780000017D701001307874762
:10303000832607000327070003A74604130717008A
:1030400023A2E6046FF09FFB03A7070083A60700F7
:10305000832747049387F7FF2322F70483A74604B7
:10306000E39207FC7360043067800000130101FFE6
:103070002326110023248100EFD0CFE597D701004C
:103080009387074103A40700EFD04FE48320C100DA
:10309000130504000324810013010101678000006F
:1030A00097D701009387073F03A5070067800000BB
:1030B000130101FD23261102232481022322910200
:1030C00023202103232E3101232C4101232A5101E6
:1030D000232861012326710197D70100938747397F
:1030E00083A70700639A070617D701001307473A1B
:1030F000832707009387170097D6010023AAF63885
:10310000832A0700638A0A0A97D7010093878736C4
:1031100083A707009304000063FEFA0A97D9010011
:103120009389094A17DA0100130ACA3783270A006C
:103130009306100003A7C70293172700B387E70081
:1031400093972700B389F90083A7090063F4F60277
:10315000930410006F00000297D701009387873215
:1031600083A70700930400009387170017D7010077
:10317000232AF73097D701009387873083A707006A
:1031800063840700930410008320C102032481029A
:103190001385040003290102832441028329C1010C
:1031A000032A8101832A4101032B0101832BC100E2
:1031B000130101036780000017D401001304442E9B
:1031C0008327040083A707006388070C737004300B
:1031D0006F00000017D401001304842C97D901005C
:1031E0009389093E17DA0100130ACA2B17DB010085
:1031F000130BCB298327040083A7070063800708EC
:103200008327040083A7C70003A9C70083274900B9
:10321000930B490013850B0063EAFA06EFD0CFDB6E
:10322000832789021305890163840700EFD0CFDA71
:103230008327C90203270B0093850B0013952700F2
:103240003305F500131525003385A9006376F700D3
:1032500017D70100232CF722EFD0CFCF83270A0006
:103260000327C90283A7C702E366F7F88327040090
:103270009304100083A70700E39407F89307F0FF77
:1032800017D701002328F71E6FF05FEA17D7010058
:103290002322F71E6FF09FE917D7010013070720BD
:1032A000832704000327070097D6010023AAE61E00
:1032B00017D701002324F71E97D701009387071C17
:1032C00083A707009387170017D701002328F71A51
:1032D0008327040083A70700639A07009307F0FF82
:1032E00017D701002328F7186FF01FE28327040087
:1032F00083A7C70083A7C70083A7470017D701008C
:10330000232AF7166FF05FE097D7010093874716DF
:1033100003A7070063160700737004306F000000F6
:10332000130101FE232E1100232C8100232A91007A
:103330002328210123263101232441012322510185
:10334000232061017370043097D401009384C41367
:1033500003A704006310071203A707001307F7FF72
:1033600097D6010023A6E61083A70700639E070AED
:1033700097D701009387071283A707006386070A80
:1033800097DA0100938ACA2317DA0100130A0A1098
:1033900017D9010013090911930910006F00C0012A
:1033A0003385EA00EFD00FBB832709000327C4024F
:1033B00083A7C7026374F70683A70A0F6380070E0B
:1033C00083A7CA0F03A4C70013058401EFD0CFC0A1
:1033D000130B440013050B00EFD00FC08327C4026A
:1033E00083260A0093050B00139527003305F5008B
:1033F00013152500130705003385AA00E3F2F6FA3A
:1034000017D701002324F708EFD0CFB48327090092
:103410000327C40283A7C702E360F7FA97D7010026
:1034200023A037076FF05FF91304000083A704009F
:10343000638C070097D701009387C70683A707000F
:1034400083A7470463980704130504008320C10180
:103450000324810183244101032901018329C1003F
:10346000032A8100832A4100032B0100130101027A
:103470006780000017D701001307C70283260700E3
:103480000327070003A746041307170023A2E60437
:103490006FF09FECEF50C06F6FF01FFB17D401006F
:1034A000130444FE83270400638C0702832704006F
:1034B0001309100063860702EFF09FBF6306050043
:1034C00097D7010023AE27FB832704009387F7FFDC
:1034D00017D701002328F7FA83270400E39E07FC8F
:1034E00097D701009387C7F903A707009307100038
:1034F000E31CF7F2EFD0CF89130410006FF01FF335
:103500006304050263960500737004306F000000C9
:1035100017D701001307C7F583270700638A070041
:10352000737004306F000000737004306F0000008F
:10353000130101FF232481002326110083260700A5
:10354000032705009386160017D601002322D6F222
:1035500097D601009386C6F383A606003304B7000E
:103560002320850063F0E6046372E40263F08602C0
:1035700097D70100938707F303A5070013054500BC
:10358000EFD08FA513050400EF500058EFF0DFD700
:10359000630E05008320C100032481001301010193
:1035A00067800000E366E4FC6FF05FFC03248100A9
:1035B0008320C100130101016FC09FFD630E050050
:1035C00017D701001307C7EA83270700638807009E
:1035D000737004306F0000006FC09FFB130101FF88
:1035E00023261100232481000327070093070500E9
:1035F0001307170097D6010023ACE6E697D6010023
:10360000938646EA17D70100130787E803270700C8
:1036100003A506003304F70013054500EFD0CF9B48
:1036200013050400EF50404EEFF01FCE631A050063
:10363000032481008320C100130101016FC05FF5E5
:103640008320C10003248100130101016780000071
:10365000130101FF232481002326110097D70100C5
:10366000938707E183A707001304000093871700DF
:1036700017D70100232EF7DE97D70100938787E144
:1036800083A7070063EEF51417DE0100130E0EFF8B
:1036900097D20100938202F2130400001307000086
:1036A000930F10001303500A6F00C000130ECEFEDC
:1036B0006384C20F83278EFF93060700E38807FE0B
:1036C0008327CEFF83A74700232EFEFE6386C71302
:1036D00003AFC70083A747003307E500930E000040
:1036E000232EFEFE6380C70983A8C7009387480383
:1036F000232017012322F70083A788042326F7013C
:103700002324F70083A7C8022328F70083A708050E
:10371000232C0700232AF70003A808038347080087
:1037200063986704930708009387170083C6070010
:10373000B3850741E38A66FE93D52500939505017D
:1037400093D50501231EB700938E1E0013070702B1
:10375000630A1F038327CEFF83A74700232EFEFEA5
:10376000E394C7F983274E00232EFEFE6FF0DFF7A8
:1037700093050000231EB700938E1E001307070257
:10378000E31A1FFD3304D40113175400130ECEFEA9
:1037900093060700E390C2F397D70100938747D0C1
:1037A00003AE070083270E006396071297D7010028
:1037B0009387C7CE03AE070083270E00639A071CCA
:1037C00017DE0100130ECEDF83274E10639C070225
:1037D00083278E11639C07266304060023200600BE
:1037E000EFF09FB2130504008320C1000324810081
:1037F000130101016780000083274E00232EFEFE87
:103800006FF01FED83278E1017DF0100130F0FECF1
:1038100083A7470017D701002328F7EA6386E73D0F
:1038200083A2C70083A74700B306D500930E00000C
:1038300017D70100232AF7E8930F40001303500A1B
:103840006382E70983A8C7009387480323A0160172
:1038500023A2F60083A7880423A6F60123A4F6007A
:1038600083A7C80223A8F60083A7080523AC060097
:1038700023AAF60003A8080383470800639A673267
:10388000930708009387170003C70700B385074114
:10389000E30A67FE93D725009397070193D70701A3
:1038A000239EF600938E1E0093860602638C1231CF
:1038B00083278E1083A7470017D701002326F7E040
:1038C000E392E7F983270E1117D70100232EF7DEC5
:1038D0006FF05FF783274E00130F8E0083A647001B
:1038E0002322DE006380E633B307E50003A746002A
:1038F00083A2C600930E00002322EE00930F200047
:103900001303500A6300EF088328C7001387480396
:1039100023A0170123A2E70003A7880423A6F70129
:1039200023A4E70003A7C80223A8E70003A708050C
:1039300023AC070023AAE70003A8080303470800F5
:10394000631E67221307080013071700834607004A
:10395000B3050741E38A66FE13D725001317070155
:1039600013570701239EE700938E1E0093870702DB
:103970006380122383264E0003A746002322EE0015
:10398000E314EFF80327CE002322EE006FF0DFF7F9
:1039900083274E00130F8E0083A747002322FE00CB
:1039A000638CE72583A2C70083A74700B306D50031
:1039B000930E00002322FE00930F20001303500AF1
:1039C0006300FF0883A8C7009387480323A016015C
:1039D00023A2F60083A7880423A6F60123A4F600F9
:1039E00083A7C80223A8F60083A7080523AC060016
:1039F00023AAF60003A80803834708006398671406
:103A0000930708009387170003C70700B385074192
:103A1000E30A67FE93D725009397070193D7070121
:103A2000239EF600938E1E0093860602638A12136D
:103A300083274E0083A747002322FE00E314FFF8EC
:103A40008327CE002322FE006FF0DFF78327CE11FD
:103A500097DE0100938ECEC883A7470017D70100D9
:103A6000232EF7C6638AD71783AFC70083A7470003
:103A70003307D5001303000097D6010023A0F6C634
:103A8000130F3000930220009308500A6388D7096F
:103A900003A5C700930745032320A7002322F700AF
:103AA000832785042326E7012324F7008327C50203
:103AB0002328F70083278502638407002326570005
:103AC00083270505232C0700232AF7000328050375
:103AD00083470800639C1705930708009387170026
:103AE00083C60700B3850741E38A16FF93D72500F5
:103AF0009397070193D70701231EF70013031300C1
:103B000013070702638EAF028327CE1183A74700F6
:103B100097D6010023A4F6BCE39CD7F783274E1267
:103B200097D6010023ACF6BA6FF09FF6930700001A
:103B3000231EF7001303130013070702E396AFFCDD
:103B400033046400E31C06C86FF09FC993070000AC
:103B5000239EF600938E1E0093860602E39A12EDD2
:103B600017DE0100130ECEA583274E103304D401B7
:103B700093165400E38E07C46FF0DFC813070000EC
:103B8000239EE700938E1E0093870702E39412DFC3
:103B900097D701009387879003AE07003304D401C1
:103BA0009316540083270E00E38C07C06FF05FDE8E
:103BB00093070000239EF600938E1E009386060254
:103BC000E39812CF83278E113304D4019316540047
:103BD000E38407C06FF09FE783274E1217D70100D9
:103BE000232EF7AE6FF05FE883270E1117D7010081
:103BF000232CF7AC6FF0DFC28327CE002322FE0018
:103C00006FF05FDA8326CE002322DE006FF0DFCD77
:103C1000130101FD2322910223202103232E3101D0
:103C2000232C4101232A51012328610123267101FC
:103C3000232611022324810297D901009389498305
:103C400017D901001309C99717DA0100130ACA83AB
:103C500097DA0100938A0A8597DB0100938B8B83A7
:103C600097D4010093844483130B10006F0000026B
:103C700083A70900032449109387170017C7010081
:103C80002328F77EEFF04FE8631E040083A70400AB
:103C9000E39007FE83270900E37AFBFEEFC05F8F06
:103CA0006FF0DFFE7370043083270A00639E070401
:103CB0008327091103A4C70013054400EFC0DFB137
:103CC00083A70B009387F7FF17C701002324F77C16
:103CD00083A704009387F7FF17C70100232EF77A05
:103CE00083270A006388070083A70A0083A7470485
:103CF0006398070203250403EF200038130504002E
:103D0000EF2080376FF09FF803A70A0083A70A000F
:103D100083274704938717002322F7046FF05FF986
:103D200003A70A0083A60A00832747049387F7FFA7
:103D30002322F70483A74604E39E07FA7360043046
:103D40006FF05FFB97C701009387877283A7070017
:103D50006396070E130101FF2326110097C7010088
:103D600023A0077217C701001307C7738327070033
:103D7000B7A6A5A59386565A83A7070383A5070070
:103D8000639ED50003A64700631AB60083A687008A
:103D90006396C60083A7C700638AD7000325070080
:103DA0008325070093854503EF30807E97C6010089
:103DB0009386C66D03A6060017D701001307478038
:103DC0006F00000283A706006382070883A706002E
:103DD0009387F7FF17C60100232AF66A03A6060099
:103DE00093172600B387C70093972700B307F70000
:103DF00083A70700E38807FC03A6060093172600A5
:103E0000B387C70093972700B305F70083A6450043
:103E100093878700B307F70083A6460023A2D50047
:103E2000638AF60283A7C6008320C10017C701007A
:103E3000232AF76613010101678000009307100031
:103E400017C70100232EF7626780000073700430EB
:103E50006F000000930740013306F60283A6460078
:103E60003307C7002322D7006FF0DFFB130101FEE9
:103E700023282101232E1100232C8100232A9100C5
:103E800023263101130905007370043097C4010023
:103E90009384845F83A7040017C401001304846023
:103EA000639C070C6314090003290400930949006B
:103EB00013850900EFC05F9283278902638607009C
:103EC00013058901EFC05F919385090017D50100A3
:103ED00013058580EFC01F8883A70400638807004F
:103EE0008327040083A747046394070A83270400F9
:103EF0006384270D83A70400638207067370043070
:103F000083A704006398070E97C70100938747595A
:103F100003A70700032707006310070C9307F0FFB0
:103F200017C701002328F75483A7040063880702FA
:103F30008327040083A74704638207020327040042
:103F400083260400832747049387F7FF2322F7047F
:103F500083A7460463940700736004308320C10183
:103F60000324810183244101032901018329C10024
:103F70001301010267800000032704008327040067
:103F800083274704938717002322F7046FF09FF1DC
:103F90000327040083260400832747049387F7FF41
:103FA0002322F70483A74604E39207F473600430E6
:103FB00083270400E39027F583A7040063820706A4
:103FC00097C701009387C74A83A707006388070A3A
:103FD000737004306F00000083A7070083A7C70039
:103FE00083A7C70083A7470017C701002324F7480A
:103FF0006FF09FF3032704008327040083274704FF
:10400000938717002322F70497C701009387474936
:1040100003A7070003270700E30207F06FF0DFFBA9
:1040200097C701009387074717C701001307475930
:1040300083A70700032787116314F7028320C101B8
:104040000324810197C7010023AE07448324410163
:10405000032901018329C1001301010267800000C7
:10406000032481018320C10183244101032901012B
:104070008329C100130101026FF0DFCC0324810109
:104080008320C10183244101032901018329C10047
:10409000130101026FC0CFCF6306050A130101FFB0
:1040A0002322910097C401009384C43F232021015F
:1040B0001389050083A50400232611002324810011
:1040C00093858501EFC00FEC03A50400130545009F
:1040D000EFC08FF09307F0FF630AF90697C701005E
:1040E0009387073B03A4070003A7040083A70700E7
:1040F0003304240123228700636EF40697C701006E
:104100009387073A03A5070083A50400938545001C
:10411000EFC04FE797C701009387C73583A7070014
:104120006376F40097C7010023A687348320C1007B
:1041300003248100832441000329010013010101AC
:1041400067800000737004306F00000083A50400D6
:10415000032481008320C10083244100032901003E
:1041600017C501001305455793854500130101014B
:104170006FC04FDE97C701009387473203A5070042
:104180000324810083A504008320C100832441000F
:104190000329010093854500130101016FC08FDEE3
:1041A000630E050097C701009387872C83A707003C
:1041B000639A0700737004306F000000737004305E
:1041C0006F000000130101FF2322910097C401003A
:1041D0009384442D03A704009387050083A504005E
:1041E000B7060080B3E7D7002326110023248100FF
:1041F000232CF7009385850113040600EFC08FD5AB
:1042000003A5040013054500EFC00FDD9307F0FF81
:104210006304F40297C701009387872703A507006B
:104220008320C100832441003305850003248100DD
:10423000130101016F40500D83A504000324810088
:104240008320C1008324410017C501001305C54820
:1042500093854500130101016FC0CFCF6308050AA4
:10426000130101FF2322910097C40100938484234A
:10427000232021011389050083A5040023261100B2
:10428000232481009385850113040600EFC08FCCA1
:1042900003A5040013054500EFC00FD493071000D9
:1042A000630AF40697C701009387871E03A40700DB
:1042B00003A7040083A707003304240123228700F7
:1042C000636EF40697C701009387871D03A5070057
:1042D00083A5040093854500EFC0CFCA97C70100AE
:1042E0009387471983A707006376F40097C70100F7
:1042F00023A287188320C100032481008324410066
:10430000032901001301010167800000737004306C
:104310006F00000083A50400032481008320C100F6
:10432000832441000329010017C501001305C53A84
:1043300093854500130101016FC0CFC197C70100EC
:104340009387C71503A507000324810083A50400F4
:104350008320C10083244100032901009385450087
:10436000130101016FC00FC2130101FF23261100C9
:1043700023248100232291008327C50003A4C700C2
:104380006304040A9304840113850400EFC0CFC4BE
:1043900097C701009387C70D83A70700639A070893
:1043A0009304440013850400EFC00FC397C70100B6
:1043B0009387C70D0327C40283A7070063F6E700AE
:1043C00097C7010023A4E70C93172700B387E700E2
:1043D0009397270017C501001305851E93850400D8
:1043E0003305F500EFC00FB797C701009387870B20
:1043F00083A707000327C4021305000083A7C70291
:1044000063FAE7009307100017C70100232AF70695
:10441000130510008320C100032481008324410080
:104420001301010167800000737004306F00000009
:104430009385040017C5010013058527EFC08FB1D0
:104440006FF09FFA97C701009387870283A7070041
:1044500063960700737004306F000000130101FFC2
:10446000232611002324810023229100B707008016
:104470000324C500B3E7F5002320F5006308040812
:10448000EFC08FB59304440013850400EFC0CFB490
:1044900097C70100938787FF0327C40283A70700FC
:1044A00063F6E70097C7010023A2E7FE93172700F2
:1044B000B387E7009397270017C501001305451040
:1044C0003305F50093850400EFC0CFA897C701001E
:1044D000938747FD83A707000327C4021305000045
:1044E00083A7C70263FAE7009307100017C701000C
:1044F0002328F7F8130510008320C100032481004E
:1045000083244100130101016780000073700430AF
:104510006F0000006304050297C70100938707F648
:1045200003A7070097C70100938787F683A70700B3
:104530002320E5002322F50067800000737004301B
:104540006F0000006304050E638E050C130101FF6C
:104550002326110023248100130705007370043003
:1045600097C80100938848F283A708006380070278
:1045700097C70100938707F383A6070083A7070067
:1045800083A746049387170023A2F60417C30100EC
:10459000130303F083A70500032603009306F0FF2F
:1045A000130400006388D70417CE0100130E0EED2C
:1045B00003250E0003280700832647006306A80092
:1045C000130410006378D6023308D6401304100099
:1045D0006372F80203250E00B387C7400326030069
:1045E000B387D70023A0F5002320A7002322C7000C
:1045F0001304000083A70800638C070097C701001D
:10460000938747EA83A7070083A7470463940702B9
:10461000130504008320C10003248100130101015C
:1046200067800000737004306F0000007370043006
:104630006F000000EF40C0556FF09FFD9307100022
:1046400017C70100232EF7E267800000630605000C
:104650000325C50467800000130500006780000083
:10466000630405002326B5046780000097C7010096
:10467000938747E303A507006780000097C7010001
:10468000938787E083A7070013051000638C07005A
:1046900097C701009387C7DD03A5070013351500F1
:1046A0001315150067800000630C0508130101FE57
:1046B000232A910097C401009384C4DE83A70400D9
:1046C000232E1100232C81002328210123263101D0
:1046D0000327C50283A7C7026376F70483278501F2
:1046E00063CC070083A7040083A6C7029307A0003A
:1046F000B387D740232CF50093172700B387E70033
:104700000327450117C90100130989EB9397270077
:10471000B307F9006308F70283A7040083A7C70261
:104720002326F5028320C101032481018324410152
:10473000032901018329C1001301010267800000E0
:1047400067800000930945001304050013850900E4
:10475000EFC08F8883A7040017C70100130707D392
:104760000327070083A7C7022326F4026376F70016
:1047700017C70100232CF7D0139527003305F50048
:1047800003248101131525008320C10183244101E5
:10479000938509003305A9008329C100032901017C
:1047A000130101026FB01FFB63060502130101FF35
:1047B00023261100232481002322910097C70100A2
:1047C000938747CE03A40700630AA40073700430E4
:1047D0006F00000013050000678000008327440578
:1047E00063960700737004306F0000008326C402D4
:1047F000032704059387F7FF232AF4046384E60064
:10480000638E0700130500008320C100032481008C
:1048100083244100130101016780000093044400D8
:1048200013850400EFB05FFB8327040517C7010061
:104830001307C7C5832607001307A0003307F740F7
:104840002326F402232CE40063F6F60017C70100C8
:10485000232EF7C213074001B387E70217C50100F3
:10486000130505D6938504003305F500EFB09FEEE0
:10487000130510006FF05FF97370043097C70100E3
:10488000938787C083A707006380070297C701004B
:10489000938747C103A7070083A70700832747041F
:1048A000938717002322F7046780000097C7010051
:1048B000938787BD83A70700638C070297C7010012
:1048C000938747BE03A70700032747046302070235
:1048D00003A7070083A60700832747049387F7FFF2
:1048E0002322F70483A7460463940700736004300F
:1048F0006780000097C701009387C7BA03A6070027
:1049000083A6070003A707009307A00083A6C6029B
:1049100003258601B387D740232CF700678000006A
:1049200097C70100938707B803A70700630A07002A
:1049300083A6070003A746051307170023AAE6046A
:1049400003A5070067800000130101FD2320210358
:10495000232611022324810223229102232E3101D6
:10496000130905007370043097C401009384C4B127
:1049700083A7040017C401001304C4B2639E070A8E
:104980008327040083A78705639A07008327040011
:104990001307100023AEE704639A050E83A70400F3
:1049A000638807008327040083A74704639A0714DA
:1049B0007370043083A70400639407068327040000
:1049C00003A5870563080500630209048327040023
:1049D00023AC07048327040023AE070483A7040045
:1049E000638807008327040083A7470463920706B0
:1049F0008320C1020324810283244102032901028E
:104A00008329C1011301010367800000032704000B
:104A1000832787059387F7FF232CF7046FF09FFB0D
:104A20000327040083270400832747049387170084
:104A30002322F7046FF09FF8032704008327040064
:104A400083274704938717002322F7046FF05FF34F
:104A50000327040083260400832747049387F7FF76
:104A60002322F70483A74604E39407F87360043015
:104A70008320C1020324810283244102032901020D
:104A80008329C1011301010367800000032504008D
:104A90002326B10013054500EFB01FD48325C100C4
:104AA0009307F0FF6380F50897C701009387479E3F
:104AB00083A907000327040083A70700B389B9006F
:104AC0002322370163ECF90697C701009387479DBE
:104AD00003A507008325040093854500EFB09FCA16
:104AE00097C701009387079983A7070063F6F9002A
:104AF00097C7010023A03799EFB09FA96FF01FEA75
:104B00000327040083260400832747049387F7FFC5
:104B10002322F70483A74604E39C07E8736004306C
:104B20006FF01FE98325040017C501001305C5BAFE
:104B300093854500EFB01FC26FF01FFC97C70100BF
:104B40009387C79503A50700832504009385450037
:104B5000EFB05FC36FF05FFA130101FD2320210363
:104B6000232E3101232611022324810223229102C4
:104B7000232C41011389050093090600737004304A
:104B800097C401009384449083A7040017C40100D4
:104B900013044491639C0714032704009307200027
:104BA0000327C7056304F702832704001345F5FFB5
:104BB00003A787053375E50023ACA704832704000A
:104BC0001307100023AEE704639A060A83A70400C4
:104BD000638807008327040083A7470463940716AC
:104BE0007370043083A70400639E0706638809007E
:104BF0008327040083A7870523A0F9000327040067
:104C000093071000130500000327C705630EF70084
:104C1000832704001349F9FF1305100003A7870534
:104C20003379E90023AC27058327040023AE07046A
:104C300083A70400638807008327040083A7470431
:104C40006392070C8320C102032481028324410262
:104C5000032901028329C101032A810113010103F0
:104C6000678000000327040083270400832747048C
:104C7000938717002322F7046FF05FF703250400E2
:104C80002326D10013054500EFB01FB58326C100D0
:104C90009307F0FF638AF60C97B701009387477F6D
:104CA00003AA07000327040083A70700330ADA00DA
:104CB000232247016368FA0C97B701009387477E68
:104CC00003A507008325040093854500EFB09FAB43
:104CD00097B701009387077A83A707006370FA0AE2
:104CE00097B7010023A847796F0040090327040004
:104CF0008327040083274704938717002322F704A0
:104D00006FF09FE9032704008326040083274704EC
:104D10009387F7FF2322F70483A74604E39407F25F
:104D2000736004308320C102032481028324410282
:104D3000032901028329C101032A8101130101030F
:104D400067800000032704008326040083274704AC
:104D50009387F7FF2322F70483A74604E39207E82B
:104D6000736004306FF0DFE78325040017C501008E
:104D70001305859693854500EFB0DF9DEFB05F8109
:104D80006FF0DFE497B701009387477103A5070031
:104D90008325040093854500EFB0DF9E6FF01FFE72
:104DA000630A050C130101FF23261100232481004F
:104DB00023229100232021017370043097B4010055
:104DC0009384846C83A704006396070863860600B7
:104DD0008327850523A0F60093070600930620008D
:104DE0000326C505232ED5041387050013040500EB
:104DF0006382D70A63F4F608930530006388B7002E
:104E0000930540006396B700630CD610232CE4048E
:104E100093071000630CF6081304100083A7040026
:104E2000638C070097B701009387C76783A70700C4
:104E300083A7470463980706130504008320C10075
:104E4000032481008324410003290100130101018F
:104E50006780000097B701009387C76403A7070026
:104E600083A7070083274704938717002322F704AB
:104E70006FF0DFF5737004306F00000093061000D0
:104E8000E398D7F88327850533E7B700232CE5049B
:104E90006FF01FF88327850593871700232CF504EF
:104EA0006FF01FF7EF30D04E6FF01FF91309440079
:104EB00013050900EFB05F9217B701001307075DF4
:104EC0008327C402032707006376F70017B70100A2
:104ED000232EF75A13074001B387E70217B50100E5
:104EE0001305056E930509003305F500EFB09F86A5
:104EF0008327840263860700737004306F0000000C
:104F000097B701009387075A83A707000327C402B6
:104F100083A7C702E3F2E7F0EFB08FE76FF0DFEFB0
:104F2000130400006FF09FEF63080508130101FEF2
:104F3000232C8100232A91002328210123263101DB
:104F40002324410123225101232E1100930907003C
:104F5000138A060093040600138905001304050054
:104F6000EFB04FF7930A050063060A008327840514
:104F70002320FA000327C40593072000232EF404FE
:104F80006380F40463FA9710930630006388D400BA
:104F9000930640006396D400630CF70E232C24057F
:104FA000930710006312F70A8327840263820702C3
:104FB000737004306F000000737004306F000000E5
:104FC0008327840593871700232CF4046FF05FFD7B
:104FD00097B701009387C74983A707006390070A23
:104FE0009304440013850400EFB00FFF17B70100CE
:104FF0001307C7498327C402032707006376F70016
:1050000017B701002324F74813074001B387E702CD
:1050100017B501001305C55A938504003305F50043
:10502000EFB04FF397B701009387C74783A70700F7
:105030000327C40283A7C70263F8E7006386090059
:105040009307100023A0F9001304100013850A0031
:10505000EFB0CFE7130504008320C10103248101D1
:1050600083244101032901018329C100032A81000E
:10507000832A410013010102678000009305840127
:1050800017B501001305C562EFB0CFEC6FF09FF9C3
:10509000130400006FF09FFB93071000E392F4F0FD
:1050A0008327840533E92701232C24056FF05FEF64
:1050B000630A050E130101FE232C8100232A9100AF
:1050C0001304050023282101232E1100232631017A
:1050D00093840500EFB00FE0930720008326C405FA
:1050E000232EF404832784051307100013090500F9
:1050F00093871700232CF4046396E6088327840221
:1051000063860700737004306F00000097B70100DA
:105110009387073683A70700639A0708930944001B
:1051200013850900EFB04FEB17B7010013070736DF
:105130008327C402032707006376F70017B701002F
:105140002326F73413074001B387E70217B50100A0
:1051500013050547938509003305F500EFB08FDF90
:1051600097B701009387073483A707000327C4027A
:1051700083A7C70263F8E700638604009307100063
:1051800023A0F400032481018320C1018324410171
:105190008329C1001305090003290101130101023C
:1051A0006FB0CFD2737004306F000000930584019C
:1051B00017B501001305C54FEFB0CFD96FF05FFAF7
:1051C00093070500630805067370043017B70100E4
:1051D0001307872B83260700639E060203A6C705D5
:1051E00093062000130500006316D60023AE0704C3
:1051F0001305100083270700638C070097B7010091
:105200009387472A03A7070003274704631C070265
:105210006780000097B601009386C62803A60600A3
:1052200083A6060083264604938616002322D6040E
:105230006FF0DFFA97B701009387C72683A70700AF
:105240006FF09FF803A7070083A607008327470492
:105250009387F7FF2322F70483A74604E39A07FA0C
:105260007360043067800000130101FB2322910466
:1052700023202105232C4103232A510323286103E2
:10528000232671032326110423248104232E3103B2
:1052900023248103232291032320A10317B90100B2
:1052A0001309492117BB0100130B0B2097B4010010
:1052B0009384C41F97BA0100938A8A1F130A1000AF
:1052C000930B90008327090003A7070063060716C6
:1052D00083A7C70083A90700EFD09FCFEFD0DFD00F
:1052E00083270B00130C05006368F50C97B70100CA
:1052F00023ACA71A130600006376352303A5040028
:10530000B3858941EFC01FA0EFE00F80630605164B
:1053100003A5040093060000130600009305810016
:10532000EFC00FAFE30005FA83278100E3C207FE59
:105330008329010183A7490163860700138549007A
:10534000EFB08FC9EFD05FCA83270B00130C0500A5
:105350006362F50C8327810017B7010023268715A8
:10536000E3E8FBFAB317FA0013F7072163100720ED
:1053700013F7770C6316072A93F70702E38A07F8F7
:1053800013850900EF00504F6FF09FF883A7C70007
:1053900003A4C70083AC07009309440013850900E8
:1053A000EFB08FC38327440213050400E780070092
:1053B0008327C4016386470D8327090003A70700DD
:1053C000E31607FC03A70A0097B6010023AE860D7B
:1053D00097B6010023AEF60C97B7010023ACE70C9B
:1053E000EFD09FF26FF0DFF283A7C70003A4C700DE
:1053F00003AD0700930C440013850C00EFB0CFBD44
:105400008327440213050400E78007008327C401B3
:10541000638C470B8327090003A70700E31607FCEB
:1054200003A70A0097B6010023A4F60897B7010066
:1054300023A2E7086FF01FF2EFD09FB9EFD0DFBAD9
:1054400083270B00130C0500E368F5F683A70A0019
:1054500003A504009309000003A60700B385894152
:1054600017B701002322870513361600EFC09F8966
:10547000EFD09FE9E31E05E8EFB08F916FF05FE991
:105480008327840193850900B387FC0063E2FC084D
:1054900083A7040063860702232A0100232C9101BD
:1054A000232E8100EFF08F9D03A5040093060000DA
:1054B0001306000093054101EFB05FAEE31E05EE59
:1054C000737004306F0000008327840193850C0003
:1054D000B307FD006362FD0883A70400638607022B
:1054E000232A0100232CA101232E8100EFF00F9924
:1054F00003A5040093060000130600009305410174
:10550000EFB0DFA9E31805F0737004306F000000FE
:10551000032509002322F40023288400EFB08FA67E
:105520006FF09FE9EFD05FDE8327090083A7C700F4
:1055300003A4C700930C440013850C00EFB0CFA95F
:105540008327C401638A47058327440213050400A7
:10555000E78007006FF0DFDB032509002322F4005A
:1055600023288400EFB00FA26FF0DFEA8327C10089
:1055700023ACF9006382070AB387870123A2F900ED
:1055800023A83901938549006362FC0803A50A003A
:10559000EFB04F9F6FF0DFD783278401232884006B
:1055A0003387F9002322E400636AEC04330C3C41A6
:1055B000636EFC0283A7040063860702232A0100AE
:1055C000232C3101232E8100EFF04F8B03A5040023
:1055D000930600001306000093054101EFB01F9CE5
:1055E000E31405F6737004306F00000003A50A0091
:1055F00093850C00EFB00F996FF01FF5032509009C
:1056000093850C00EFB00F986FF01FF4032509008D
:10561000EFB04F976FF0DFCF737004306F00000072
:105620008327C10083A6890123A839013387D700C6
:1056300023A2E9006362EC06B307FC4063EAD706E5
:1056400083A7490213850900E780070083A7C901E2
:10565000E39047CD83A689018327C10003A70400F7
:10566000B387D70063060702232A0100232CF10029
:10567000232E3101EFF08F8003A504009306000074
:105680001306000093054101EFB05F91E31205C8D6
:10569000737004306F0000006374FC00E372F7FA6B
:1056A0000325090093854900EFB0CF8D6FF05FC6E9
:1056B00003A50A0093854900EFB0CF8C6FF05FC55A
:1056C000130101FF232481002326110023229100CE
:1056D0002320210117B40100130444DDEFF0CF991A
:1056E0008327040063840704EFF04F9C83270400A2
:1056F000638A070293080000130800009307000064
:1057000013072000930600001306004097B5010020
:105710009385C5CA17050000130545B5EFC0DF9E88
:1057200063140506737004306F00000017B90100A0
:105730001309C9FB13050900EFA05FFF97B401002F
:10574000938404FC13850400EFA05FFE13060000A1
:105750009305C0001305400097B7010023AC27D57F
:1057600097B7010023A697D4EFB04FCA17B701002F
:10577000232EA7D26306050297B50100938585C342
:10578000EFC00FC56FF05FF68320C10003248100D6
:1057900083244100032901001301010167800000F7
:1057A000737004306F000000638A050A130101FD65
:1057B000232A5101930A05001305C0022324810204
:1057C0002322910223202103232E3101232C410186
:1057D00023261102232861012326710113090700E2
:1057E00093890600130A060093840500EF00C07039
:1057F00013040500630C0502EFF00F8897B7010052
:105800009387C7CA83A70700638E0704EFF00F8A48
:105810001305440023205401232C9400232E44011B
:105820002320340323222403EFA05FF21305040096
:105830008320C1020324810283244102032901023F
:105840008329C101032A8101832A4101032B01011C
:10585000832BC100130101036780000073700430C3
:105860006F00000097BB0100938B4BE813850B0082
:10587000EFA0DFEB17BB0100130B8BE813050B0048
:10588000EFA0DFEA130600009305C00013054000F7
:1058900097B7010023A077C397B7010023AA67C178
:1058A000EFB0CFB617B701002322A7C0630A0500E7
:1058B00097B50100938505B0EFC08FB16FF01FF56C
:1058C000737004306F000000630E0506130101FEC3
:1058D000232C8100232E1100232A910017B40100EC
:1058E0001304C4BC8328040013080500130500003A
:1058F00063800804930407002322B1001387060085
:105900002324C100232601019306500063C0B6047E
:10591000EFE0DFD693072000630EF50403250400B3
:10592000930600001306000093054100EFB00FE757
:105930008320C10103248101832441011301010259
:1059400067800000737004306F0000009305410011
:10595000930600001306070013850800EFB0DF99D7
:105960008320C10103248101832441011301010229
:1059700067800000032504009306000013860400DE
:1059800093054100EFB08FE16FF09FFA63060500C9
:105990000325050067800000737004306F0000006D
:1059A00063160500737004306F000000130101FFDF
:1059B000232611002324810013040500EFE0DFEB10
:1059C000032544013334A000EFE05FEE130504002B
:1059D0008320C100032481001301010167800000BE
:1059E00063160500737004306F000000130101FF9F
:1059F000232481001304050023261100EFE0DFE7D4
:105A000003240402EFE09FEA8320C1001305040091
:105A10000324810013010101678000006316050063
:105A2000737004306F000000130101FF2324810014
:105A300023229100138405009304050023261100FE
:105A4000EFE09FE323A08402032481008320C100B0
:105A500083244100130101016FE05FE5130101FFA1
:105A60001305C0012324810023261100EF00C04844
:105A700013040500630805002320050013054500F5
:105A8000EFA0DFCA130504008320C10003248100B6
:105A9000130101016780000063020502B70700FFE0
:105AA000B3F7F50063860700737004306F000000E1
:105AB000639A0500737004306F0000007370043047
:105AC0006F000000130101FE232C81002328210117
:105AD000232631012324410123225101232E1100C9
:105AE000232A91009309070013890600930A0600F0
:105AF00013840500130A0500EFE05FB86318050082
:105B000063860900737004306F000000EFD04FCC43
:105B100083240A00B37794006312090463820704A4
:105B200063880A009347F4FFB3F797002320FA0035
:105B3000EFD08FFD8320C101032481011385040070
:105B400003290101832441018329C100032A810023
:105B5000832A41001301010267800000E302F4FC84
:105B6000E38809FCB335500193958501630609006C
:105B7000B7070004B3E5F50013860900B3E5850017
:105B800013054A00EFE0CFE1EFD00FF863140500F2
:105B9000EFA01FA0EFE01FD6931765009309050043
:105BA00063DA0700B70400019384F4FFB3F49900AB
:105BB0006FF05FF8EFE05FCC83290A00B377340120
:105BC00063100902638A070063880A009347F4FFA1
:105BD000B3F737012320FA00EFE05FCD6FF09FFCB1
:105BE000E31CF4FE6FF05FFE630C0500B70700FFD7
:105BF000B3F7F500638A0700737004306F0000008C
:105C0000737004306F000000130101FF2324810032
:105C100013040500232611002322910023202101D3
:105C200013890500EFE05FC5832404009345F9FF65
:105C3000B3F795002320F400EFE05FC78320C10095
:105C400003248100138504000329010083244100FB
:105C50001301010167800000130101FF232481006B
:105C60001304050023261100EFA0DFA6032404007F
:105C7000EFA0DFA58320C1001305040003248100E9
:105C80001301010167800000630C0500370700FF66
:105C9000B3F7E500638A0700737004306F000000FB
:105CA000737004306F0000006F205071B70700FF61
:105CB000B377F60063860700737004306F0000004E
:105CC00063160600737004306F000000130101FEBC
:105CD000232C810023282101232631012324410183
:105CE000232E1100232A91001389060093890500B1
:105CF000130A050013040600EFE05F98631E050415
:105D000063060900737004306F000000EFD04FACE1
:105D100083240A009385090013050A00B3E499005F
:105D2000EFF09FF6B3779400630AF40883240A0027
:105D3000EFD08FDD8320C10103248101138504008E
:105D400003290101832441018329C100032A810021
:105D50001301010267800000EFD08FA783240A009F
:105D60009385090013050A00B3E43401EFF0DFF175
:105D7000B3F7840063848704E30A09FAB7050005D2
:105D800013060900B365B40013054A00EFE04FC1E4
:105D9000EFD08FD763140500EFA08FFFEFE09FB522
:105DA000931765009304050063D40702B707000149
:105DB0009387F7FFB3F4F4006FF0DFF783270A004F
:105DC0001344F4FFB3F787002320FA006FF05FF667
:105DD000EFE09FAA83240A00B377940063988700BA
:105DE0009347F4FFB3F797002320FA00EFE01FACCE
:105DF0006FF0DFFB130101FF232481002326110034
:105E00001304050023229100EFD08F9C83274400C8
:105E100063860702032504019304C40063189500F8
:105E20006F0080030325040163089502B705000293
:105E3000EFE04FE183274400E39607FE13050400DB
:105E4000EF008023032481008320C10083244100CC
:105E5000130101016FD04FCB737004306F0000004D
:105E6000630C0500370700FFB3F7E500638A0700FE
:105E7000737004306F000000737004306F00000016
:105E80006F20D053630C0500B70700FFB3F7F50090
:105E9000638A0700737004306F0000007370043071
:105EA0006F000000130101FF2324810023229100D1
:105EB000232611001304050093840500EFE0DF9B07
:105EC0000327040093C7F4FFB377F7002320F400FF
:105ED000032481008320C1008324410013010101B8
:105EE0006FE0DF9C630605000325850167800000E5
:105EF0001305000067800000130101FF23248100C7
:105F00002326110013040500EFD08F8C97A7010002
:105F10009387875A83A70700639C0704B7970100FC
:105F200017A701001307477F9387C7FF97A60100B4
:105F300023AAE65817A701002324F75817A7010042
:105F4000232EF77C97A701009387475717A70100D7
:105F50002324F77C9307100017A701002326075678
:105F600017A70100232C075417A701002326F75475
:105F700063120402EFD04FB9EF10C06013040000A9
:105F8000130504008320C1000324810013010101D3
:105F90006780000013058400937735006398070C31
:105FA000B79701001307F5FF9387A7FFE3E4E7FC2A
:105FB00097A601009386065183A706006F00400153
:105FC00003A70700630A07009386070093070700EB
:105FD00003A74700E366A7FE17A701001307074EB4
:105FE000E38AE7F803A7070013060001138487007C
:105FF00023A0E60003A74700B306A740637ED602AE
:106000003388A7002322D80023A2A70083254800B5
:1060100097A601009386064B6F0080009306070049
:1060200003A7060003264700E36AB6FE2320E80024
:1060300023A0060103A7470097A701009387874C79
:1060400083A70700B387E74017A70100232CF74A6F
:10605000EFD08FABE30204F2130504008320C100EC
:106060000324810013010101678000001375C5FF3F
:10607000130545006FF0DFF263080506130101FF09
:10608000232481002326110013040500EFC05FF4D0
:10609000930584FF0326C4FF17A701001307874257
:1060A0006F008000138707008327070083A647003F
:1060B000E3EAC6FE232CF4FE2320B70097A70100D5
:1060C0009387474403A707008327C4FF0324810065
:1060D0008320C100B387E70017A701002324F742FC
:1060E000130101016FD04FA26780000097A7010044
:1060F0009387474103A50700678000006780000081
:106100003367B50013773700930705006312070460
:106110009308D6FFB3081501130705009386050001
:106120006378150303A8060013074700938646000B
:10613000232E07FFE36817FF9347F5FFB387170187
:1061400093F7C7FF93874700B385F500B307F500C2
:106150003306C50063F4C70C9386450013884700D7
:10616000B3B6D70033B8050133E7F50093C6160080
:106170001348180013773700B3E6060113371700EA
:106180003377D700330EF64093861700630807066F
:106190001337AE006314070613532E00138805004F
:1061A00093860700130700008328080013071700D1
:1061B0001308480023A0160193864600E36667FE95
:1061C0001377CEFFB385E500B387E7006306EE04DF
:1061D00083C60500138717002380D700637EC7029C
:1061E00083C6150013872700A380D7006376C702F4
:1061F00003C725002381E70067800000B307F6404E
:10620000B387F5009385150003C7F5FF9386160045
:10621000238FE6FEE398F5FE6780000067800000AC
:10622000B367C50093F73700B308C5006382070E54
:1062300063761511B307A04093F737001387370033
:106240009306500093F5F50F130815003383A8400B
:106250001306F6FF6374D700130750006368E60E59
:106260006380070E2300B50013071000638EE7005C
:10627000A300B50013073000130825006396E7005C
:10628000130835002301B5001396850033E6C500D9
:10629000139705013367E6003303F34093968501B6
:1062A000B366D70013562300B307F50013070000A9
:1062B00023A0D7001307170093874700E36AC7FEA0
:1062C0001377C3FFB307E8006300E3082380B70038
:1062D00013871700637C1703A380B7001387270079
:1062E000637617032381B7001387370063701703A2
:1062F000A381B70013874700637A17012382B70091
:106300001387570063741701A382B70067800000EA
:1063100093F5F50F13978500B365B7001397050143
:106320003367B700E37415FF9307050093874700B1
:1063300023AEE7FEE3EC17FF6780000067800000F4
:10634000130805006FF05FF46780000093070500F5
:106350006FF0DFF78347050013070500638C070024
:106360001305150083470500E39C07FE3305E54050
:10637000678000001305000067800000130515000A
:106380008347F5FF9385150003C7F5FF6388070072
:10639000E386E7FE3385E74067800000930700004F
:1063A0006FF05FFF930705009385150003C7F5FFA6
:1063B00093871700A38FE7FEE31807FE67800000AE
:1063C00083460500930700026398F6001305150045
:1063D00083460500E38CF6FE938756FD93F7D70FAF
:1063E0006380070493070500930500006388060493
:1063F0001305000093871700138606FD1317250069
:1064000083C607003305A700131515003305A60042
:10641000E39206FE638405003305A0406780000018
:10642000938536FD8346150093B515009307150037
:10643000E39006FC130500006FF0DFFD130500007C
:106440006780000083A705002380A70083A70500BD
:106450009387170023A0F5006780000097A601002E
:106460009386C60683A70600173703001307872DF8
:1064700013861700B307F7002380A70097A5010034
:1064800023A6C5049307A000630AF5009307000440
:106490006308F6001305000067800000E30C06FEA9
:1064A000370610F0130717008347F7FF2320F6F095
:1064B00083A706009387F7FF97A5010023A8F5009F
:1064C000E39207FE1305000067800000130101EB53
:1064D0002322911423202115232A511323248113CD
:1064E0002326111423248114232E3113232C41132A
:1064F0002328611323267113232291132320A11330
:10650000232EB11193040500138905002326C10031
:10651000130C5002930A9000834709006388870395
:10652000638C070603A404006F00800063860706DF
:106530002300F40003A40400130919001304140039
:1065400023A0840083470900E39287FF03461900D4
:106550009308190093860800130D00029309F0FFB9
:10656000130AF0FF13080000130550059307D6FD2A
:1065700093F7F70F13891600636EF53A17A701001A
:10658000130747A893972700B387E70083A707005F
:10659000B387E700678007008320C11403248114B8
:1065A00083244114032901148329C113032A81136D
:1065B000832A4113032B0113832BC112032C811255
:1065C000832C4112032D0112832DC11113010115DA
:1065D00067800000930C80002324010093071000C3
:1065E00063DA071D8327C10003A40400938B77009F
:1065F00093F68BFF03AB060083A9460093878600C2
:106600002326F10013860C009306000013050B00EF
:1066100093850900EF20400E2328A1009307000076
:1066200063803733930D4101930B100013860C00E8
:106630009306000013050B0093850900EF109048A6
:106640009306000013860C00130B050093890500C8
:10665000EF20800A8327810023A0AD0093861B00D2
:10666000938D4D0063863701938B06006FF01FFCFE
:10667000E37C9BFF63D24603930704002380A701BA
:1066800003A40400130AFAFF9307140023A0F400E4
:1066900013840700E3C446FF93962B009307010180
:1066A000B386D7006F008002938777052300F4003C
:1066B00003A40400938BFBFF93871B0013041400B7
:1066C00023A084009386C6FFE358F0E483A7060066
:1066D000E3ECFAFC938707036FF05FFD83A70400E8
:1066E000930600030327C1002380D70083A704007B
:1066F00093064700930C00011386170023A0C400E3
:1067000013068007A380C70003A40400232401000C
:10671000930707001304140023A0840003AB0700B1
:10672000930900002326D1006FF0DFED8327C1001D
:1067300083AC0700938B470063880C28635C40257B
:106740009307D002631EFD2083C70C0063880702F5
:1067500063D8092483A60400938C1C00130AFAFF53
:106760002380F60003A404001304140023A0840073
:1067700083C70C00E39E07FC6352400303A404009C
:10678000930700022300F40003A40400130AFAFF95
:106790001304140023A08400E3160AFE23267101CB
:1067A0006FF09FD72324010093071000930CA000E3
:1067B000E3CA07E38327C10003A4040093864700CC
:1067C0006FF0DFF503C61600930609006FF01FDABD
:1067D00083A70400930650022380D70003A404007B
:1067E0001304140023A084006FF01FD3930C000146
:1067F000232401006FF09FDE8327C10003C616002B
:106800009306090083A90700938747002326F10018
:10681000E35E0AD4138A09009309F0FF6FF01FD5D5
:1068200003C61600130DD002930609006FF01FD4A3
:106830009347FAFF93D7F74103C61600337AFA005D
:10684000930609006FF09FD203C61600130D0003D4
:10685000930609006FF09FD183C51600930906FDCA
:1068600093060900938705FD13860500E3E2FAFA13
:1068700093972900B38937019386160093991900DD
:10688000B389B90083C50600938909FD938705FD87
:1068900013860500E3FEFAFC6FF09FF70327C100A3
:1068A00083A7040083260700130747002326E1007F
:1068B0002380D70003A404001304140023A0840041
:1068C0006FF09FC59307100063D4070F8327C100A3
:1068D0009386770093F686FF938786002326F10040
:1068E00083A9460083A7060063DE090E83A6040081
:1068F0001306D002B307F0402380C60003A40400AF
:10690000B336F000B30930411304140023A084000F
:10691000138B0700B389D940930CA00023240100F6
:106920006FF05FCE03C61600130818009306090027
:106930006FF0DFC383A70400138908006FF09FE99D
:10694000E3729BCF93071000930B00009306100097
:10695000E3C447D36FF05FD497AC0100938C8CA64F
:106960009385090013850C00EF10004E330AAA40EE
:106970006352400303A404002300A40103A4040001
:10698000130AFAFF1304140023A08400E3160AFE7E
:10699000130A000083C70C00E38207E0E3CC09DAA6
:1069A0009389F9FF1307F0FFE396E9DA6FF0DFDC74
:1069B0008327C1009386470083A707002326D100C1
:1069C00093D9F7416FF05FF2635640019307D0020D
:1069D000E314FDF897AC0100938CCC9E93078002E2
:1069E0006FF01FD7138B0700930CA0002324010026
:1069F00003A404006FF01FC1130101EB232E311318
:106A0000B70900409387F9FF2324811423229114AE
:106A1000232C4113232A511323261114232021153B
:106A20002328611323267113232481132322911316
:106A30002320A113232EB111130A05002324B10032
:106A400017A40100130484A8973A0300938A8ACFFD
:106A500097940100938484702326F10093055002DB
:106A60001305A00013080004B70610F083470A00BE
:106A7000638EB7046388070A03270400130A1A0009
:106A8000130617003387EA0097A8010023A0C8A4C3
:106A90002300F7006380A708E31A06FD17370300F9
:106AA000130747CA130717008347F7FF23A0F6F021
:106AB000832704009387F7FF17A601002328F6A079
:106AC000E39207FE83470A00E396B7FA83461A006B
:106AD00013051A0013070500930B0002130BF0FFB8
:106AE000130CF0FF13080000930550059308900065
:106AF0009387D6FD93F7F70F130A170063ECF5445D
:106B000093972700B387970083A70700B387970061
:106B100067800700173703001307C7C2E31406F89E
:106B20006FF0DFF48320C114032481148324411403
:106B3000032901148329C113032A8113832A4113D2
:106B4000032B0113832BC112032C8112832C4112BE
:106B5000032D0112832DC11113010115678000005F
:106B6000930C8000130D00009307100063DA0721D7
:106B7000832781009387770093F787FF83AD070012
:106B800003AB4700138787002324E10013860C0022
:106B90009306000013850D0093050B00EF10D03510
:106BA0002328A10063086D451309410193091000D2
:106BB00013860C009306000013850D0093050B004F
:106BC000EF10407013860C0093060000930D050033
:106BD000138B0500EF1050322320A9009389190070
:106BE00013094900E3166DFDE3F49DFD130600044F
:106BF000B70610F063D489038327040013871700B6
:106C0000B387FA0097A5010023A2E58C23807701C2
:106C1000630AC706130CFCFFE3C089FF8327C1008A
:106C20001305C10093089000B386F90093962600DF
:106C300093070101B386D7001308A00013030004D3
:106C4000370610F0E38CA6E083A706009305000347
:106C500063F4F8009305700503270400B387B700B9
:106C6000930517003387EA0017AE01002320BE8684
:106C70002300F70063860737638C65329386C6FF6F
:106C80006FF05FFC173703001307C7AB130717003C
:106C90008347F7FF23A0F6F0832704009387F7FFCD
:106CA00097A5010023A4F582E39207FE130CFCFFD5
:106CB0006FF09FF683270400130600041387170064
:106CC00097A5010023A4E580B386FA00930500038D
:106CD0002380B6006308C75093872700979601006A
:106CE00023A6F67E3387EA00930680072300D700A9
:106CF00017370300130707A5B70610F06392C70202
:106D0000130717008347F7FF23A0F6F0832704003B
:106D10009387F7FF17960100232AF67AE39207FE7E
:106D200083278100930C0001130D00009387470017
:106D300003278100130B0000832D07002324F1009B
:106D40006FF0DFE48327810083AC070013894700DD
:106D5000638E0C4C6358802B9307D0026394FB3EE8
:106D600003C70C00930507006314072A6F00002F68
:106D700093071000930CA000130D0000E3CA07DF77
:106D800083278100938747006FF09FFA8327810054
:106D90008346170013070A0003AB070093874700D9
:106DA0002324F100E3560CD4130C0B00130BF0FF5B
:106DB0006FF01FD483461700930BD00213070A000D
:106DC0006FF01FD39347FCFF93D7F741834617001B
:106DD000337CFC0013070A006FF09FD18346170035
:106DE000930B000313070A006FF09FD003461700B0
:106DF000138B06FD13070A00930706FD9306060092
:106E0000E3E2F8FA93172B00B38767011307170023
:106E100093971700B387C70003460700138B07FD3E
:106E2000930706FD93060600E3FEF8FC6FF09FF75C
:106E300083258100832704001306A00003A7050013
:106E400093861700B387FA00179501002320D568B1
:106E50002380E700138945006300C73693070004C9
:106E60006384F62A232421016FF05FBF930710008B
:106E700063DE07358327810013877700137787FF49
:106E8000930787002324F100032B47008327070083
:106E900063560B3E032704001306000493061700F5
:106EA0009795010023A4D5623387EA009305D002A9
:106EB0002300B700638CC638B307F0403337F000C7
:106EC000330B6041938D0700330BEB40930CA00014
:106ED000130D00006FF09FCB8346170013081800B6
:106EE00013070A006FF0DFC08346170013070A007C
:106EF0006FF01FC083270400930600041387170058
:106F0000179601002324E65CB387FA0013065002AB
:106F10002380C700E314D7B4173703001307878211
:106F2000B70610F0130717008347F7FF23A0F6F00A
:106F3000832704009387F7FF179601002328F6584C
:106F4000E39207FE6FF09FB1930C0001130D000058
:106F50006FF09FC18327040093060004130A050005
:106F600013871700179601002322E656B387FA000D
:106F7000130650022380C700E312D7AE1727030081
:106F80001307477CB70610F0130717008347F7FF76
:106F900023A0F6F0832704009387F7FF17960100DC
:106FA0002326F652E39207FE130A05006FF01FAB8B
:106FB0001727030013070779130717008347F7FF05
:106FC0002320F6F0832704009387F7FF97950100AD
:106FD00023AEF54EE39207FE9386C6FF6FF09FC681
:106FE0001727030013070776E39805FC9386C6FF6F
:106FF0006FF05FC5E3FA9DBB930910006FF01FBFF0
:10700000130C000003C70C0093050700E30C07E412
:107010009308F0FF1305A00013080004B70610F052
:10702000635E0B0C8327040013861700B387FA00F6
:1070300017930100232CC3482380E7006382A5082F
:107040006308060B938C1C0003C70C00130CFCFF99
:1070500093050700E31607FCE35680E1832704004D
:107060009305000213060004B70610F06F00C0007D
:10707000130CFCFFE3080CDE13871700B387FA003C
:107080002380B700179501002322E54493070700EA
:10709000E310C7FE172703001307C76A130717007B
:1070A0008347F7FF23A0F6F0832704009387F7FFB9
:1070B00017950100232CF540E39207FE6FF05FFB6C
:1070C0001727030013070768E30E06F613071700D8
:1070D0008347F7FF23A0F6F0832704009387F7FF89
:1070E000179601002324F63EE39207FE6FF09FF50A
:1070F00017270300130707656FF05FFD130BFBFFF6
:10710000E3121BF36FF05FF5172703001307876384
:10711000B70610F0130717008347F7FF23A0F6F018
:10712000832704009387F7FF179601002320F63A80
:10713000E39207FE232421016FF05F92979C0100E8
:10714000938C4C2893050B0013850C00EF00D04F57
:10715000330CAC40E35880EB832704001306000493
:10716000B70610F06F00C000130CFCFFE30A0CE838
:1071700013871700B387FA002380770197950100E2
:1071800023A6E53493070700E310C7FE1727030083
:107190001307475B130717008347F7FF23A0F6F099
:1071A000832704009387F7FF9795010023A0F5320A
:1071B000E39207FE6FF05FFB172703001307875862
:1071C000E39806F4232421016FF05F89832781006F
:1071D0001387470083A707002324E10013DBF7414F
:1071E0006FF01FCB172703001307C755B70610F022
:1071F000130717008347F7FF23A0F6F08327040047
:107200009387F7FF179601002322F62CE39207FEDF
:107210009307100017970100232AF72A9307800786
:10722000172703002300F7526FF09FAF63568001CA
:107230009307D002E394FBF0979C0100938C8C1889
:1072400013078002930580026FF09FDC97260300EE
:107250009386464F370610F09386160003C7F6FF55
:107260002320E6F0032704001307F7FF979501009A
:1072700023AEE524E31207FE6FF01FC4938D0700D1
:10728000930CA000130D00006FF05F90B70710F093
:1072900023A0A7F26F000000130101FC13034102B9
:1072A0002322B10293050300232E11002324C102DF
:1072B0002326D1022328E102232AF102232C0103F1
:1072C000232E110323266100EFF00FF38320C10169
:1072D000130500001301010467800000130101FB86
:1072E00013038103232481022326A100232CC1023E
:1072F00013040500130603001305C1002326110221
:107300002322F104232ED1022320E10423240105AA
:1073100023261105232E6100EFF04F9B8327C10028
:10732000238007000325C1008320C1023305854067
:10733000032481021301010567800000B70710F0E4
:1073400083A647F403A607F403A747F4E31AD7FE7E
:10735000B7160000938606FAB306D60033B6C60009
:10736000B305E60023A4D7F423A6B7F46780000092
:10737000B70710F003A747F403A607F483A647F462
:10738000E31AD7FEB7160000938606FAB306D600B6
:1073900033B6C60023A4D7F4B305E60023A6B7F49A
:1073A0009307000873A0473067800000130101FFB6
:1073B0002324810023261100130440011304F4FF49
:1073C000EF001002E31C04FE8320C10003248100AF
:1073D0001301010167800000130101FF23248100D4
:1073E00023261100979701009387C70E1794010079
:1073F0001304040E03A70700832704001306F07C80
:1074000093064706938747069795010023A4D50C5A
:107410009795010023AEF50A634AD6008320C10088
:1074200003248100130101016780000013074789CD
:107430009797010023A0E70AEF00406C9307100024
:107440006316F50203270400B71700009387F77649
:1074500013050000E3D4E7FCEFF05FE303248100B1
:107460008320C100130101016FB09FB51795010082
:107470001305C5F5EFF05FE213052000EFF01FE103
:10748000032481008320C100130101016FB05FB3A9
:1074900017950100130505F56FF01FE01795010022
:1074A0001305C5F46FF05FDF130101FF2324810092
:1074B0002322910023261100B71400001794010025
:1074C000130444F393878438130000009387F7FF75
:1074D000E39C07FE13050400EFF01FDC6FF09FFE36
:1074E000130101FF2326110023248100EF0080589F
:1074F000170700001307C7EB9306000013061000E0
:107500009305200317950100130545EFEFE0CFA980
:1075100013040500EFB05FAD13060500130504006A
:10752000032481008320C10013070000930600009C
:1075300093051000130101016FE00FB9130101FF62
:1075400023261100EF00805B130710009307000053
:10755000631AE5008320C1001385070013010101B0
:107560006780000017950100130545E6EFF0DFD2B4
:107570008320C10093072000138507001301010138
:1075800067800000737004306F00000067800000A7
:10759000737004306F000000130101FB232291047B
:1075A00023202105232E3103232C4103B73900006A
:1075B000375AC64137890000B7040100232A510316
:1075C00023286103232671032324810323229103AB
:1075D0002320A103232EB101232611042324810497
:1075E000232601001307C100979C0100938C8CF0A7
:1075F000172C0300130C0C19979B0100938B0BEFB6
:10760000179D0100130D4DEE972D0300938D0D1E58
:10761000130ADAE6938999031309F9FF130B300073
:107620009384F4FF930A10011304100033074703F7
:10763000930600001306F0FF9305C10033073701DE
:1076400093570701B3F72701B3F7670317950100B5
:107650002322E5EA93972700B307FC0003A7C7009E
:1076600003A507001307170023A6E700EF901F9359
:10767000630685009797010023AE07E88327C100C2
:10768000938717006382970603A70B002326F10058
:107690009307170017970100232AF7E463F2FA060D
:1076A00083270D0017970100232207E4638C8706C8
:1076B000638C0704130720006394E70497270300F3
:1076C0009387871203A5070093051000EFB08FA0E2
:1076D0001305800C9797010023A807E0EFB01FEE79
:1076E00003A70C006FF05FF483A70B0023260100B3
:1076F0009387170017970100232AF7DEE3E2FAFACF
:1077000003A70C006FF09FF203A50D009305000086
:10771000EFB04F9C03A70C009797010023A687DCCE
:107720006FF09FF003A50D0093051000EFB08F9A46
:10773000972703009387470B03A5070093050000D5
:10774000EFB04F999307200017970100232EF7D829
:1077500003A70C006FF05FED130101FC130590000F
:10776000232C8102232A910223282103232631037B
:1077700023244103232E11022322510323206103DA
:10778000232E7101232C8101232A91012328A10199
:1077900023260100972403009384C4FEEFA0CFF0BA
:1077A0009797010023AEA7D413890400172A03007A
:1077B000130A0AFE17940100130484D493091000DD
:1077C000130600009305400013053000EF900FC42E
:1077D0002320A900630A052483250400EFA0CFF825
:1077E000630A35239797010023A607D2130949009E
:1077F000E31849FD03A5040093050000EFA00FFD69
:10780000630605009797010023A607D0832504008F
:1078100003A50400EFA08FFB930710006306F5009B
:107820009797010023A807CE03A504009305C10084
:107830009306000013060000EF904FF68325040026
:1078400003A50400EFA04FF263060500979701001F
:1078500023A207CC03A50400930600001306000032
:107860009305C100EF90DFDA8325040003A504002F
:10787000EFA08FEF930710006306F50097970100C4
:1078800023AA07C8032504009305800CEFA04FF935
:10789000630605009797010023AE07C697270300EC
:1078A000938787F403A50700B70401003709FFFF9A
:1078B000EFB08F9C930710009389E4FF179C0100A1
:1078C000130CCCC4179A0100130ACAC417970100FD
:1078D0002324F7C2979B0100938B8BC1179D010056
:1078E000130DCDC1130B1000930A5000930C6000D0
:1078F000130919009384F4FF13050000EFA09FF013
:1079000063080506032504009305F0FFEFA04FF17F
:10791000630A050693060000130600009305C100E4
:10792000EF901FCF630665019797010023A407BE60
:10793000EFC09FF48327C10063FCF904338727015C
:1079400063F0EA02130780FF636CF70003270C0063
:107950006374F70EB387E74013073000636AF70CD0
:1079600083270A0063980708737004306F000000D3
:10797000032504009305F0FFEFA08FEAE31C05F850
:107980006FF09FF79797010023A607B86FF0DFF617
:1079900063F0FA023387F94063FCEC0003A70B00A5
:1079A0006376F70AB387E740130730006360F70C8C
:1079B00083270A0063960700737004306F0000008D
:1079C00083A70B009387170063FCF90897970100C2
:1079D00023A007B2EFC09FED83270A00E39E67F163
:1079E00083270D0093871700179701002328F7B00E
:1079F0006FF09FF083270C00938717001797010003
:107A00002326F7B0E39807FC9797010023A097B0CF
:107A10006FF05FFC0325090083250400EFA0CFD49D
:107A2000E30605DC6FF01FDC737004306F000000AC
:107A3000737004306F000000B307F7401307300085
:107A4000E370F7F2737004306F000000B307F74083
:107A500013073000E37EF7F4737004306F0000000A
:107A6000179701002326F7A86FF0DFF67370043034
:107A70006F000000130101FF9308000013080000CD
:107A800097270300938747D613071000930600003B
:107A90001306004097950100938585971705000010
:107AA0001305C5AF2326110023248100EFA0CFE5E5
:107AB00017240300130444D3832604009308000012
:107AC0001308000097270300938747D2130710007D
:107AD0001306004097950100938505941705000053
:107AE0001305C5C7EFA04FE203250400032481005E
:107AF0008320C100130101016FC04FB79727030016
:107B0000938747C8179301001303439F83A8C700B7
:107B100003A68701179701001307C79C032E0300D4
:107B20000325070003A8070183A6C70183A5470112
:107B300003A707023386C840979701009387879D64
:107B4000832E03003305C54183A707003336C000E9
:107B50003306C040B38606413335A0003375C500F7
:107B6000B336D0003307B740179301001303439A8D
:107B7000179601001306C696B306D0403337E000CF
:107B80009387F7FF032E0300032606003307E04028
:107B90003375D50093B717003375E500B307F04090
:107BA000179701002320D79517270300232817BF15
:107BB00017270300232607BF172703002324B7BE78
:107BC0003375F500630ACE00832703001797010081
:107BD0002328F790678000001305000067800000ED
:107BE000130101FE9797010093870791232E11003F
:107BF000232C810003A4070093071000630AF400FC
:107C00008320C10103248101130101026780000068
:107C1000979701009387878C83A707001307400677
:107C200093871700636EF7008320C101032481014D
:107C3000179701002324F78A1301010267800000CF
:107C4000979701009387C78B03A5070097970100BB
:107C500023A60788EFA08FBF63080508130600005E
:107C60009305C100EF901FC363068500979701003D
:107C700023A2078A8327C100370701001307E7FF04
:107C80006378F70E3707FFFF130717003387E70006
:107C90009306500063F0E616130780FF97960100E5
:107CA0009386C686636CF71403A706006374F71601
:107CB000B387E740130730006372F7147370043022
:107CC0006F00000083A70600938717001797010035
:107CD000232EF782639A0700B70701009387F7FF07
:107CE000179701002324F782178401001304C47E30
:107CF0008327040093060000130600001397270053
:107D000097270300938707A8B387E70003A5070019
:107D1000978501009385C57FEF900FDE93071000D4
:107D2000E310F5EE178701001307877E832707000E
:107D3000938717009786010023ACF67C8327070002
:107D4000639A0700B70701009387F7FF17870100C1
:107D50002320F77C83270400130720009387170054
:107D60006354F7089787010023A807766FF05FE94F
:107D70009306500063FAF6023307F740930660005B
:107D800063F4E602978601009386867603A70600D1
:107D9000637CF708B387E74013073000637AF70086
:107DA000737004306F00000097860100938646745C
:107DB000978701009387077683A7070063820702EE
:107DC00083A70600370701001307E7FF9387170013
:107DD0006376F7069787010023AC07706FF0DFF03A
:107DE000737004306F000000178701002326F76EC0
:107DF0006FF01FE197860100938646719787010017
:107E00009387477183A70700E39E07EA73700430E6
:107E10006F000000B307F74013073000E370F7FE70
:107E2000737004306F000000B307F7401307300091
:107E3000E370F7F8737004306F00000017870100DB
:107E40002328F76A6FF05FEAB305B50093070500D2
:107E50006386B70003C70700631607003385A74092
:107E600067800000938717006FF09FFE9308000063
:107E700063DC05003305A040B337A000B305B04074
:107E8000B385F5409308F0FF63DA06003306C0407F
:107E9000B337C000B306D040B386F64013080600DF
:107EA00013830600930705001387050063980624D3
:107EB000978601009386064063F8C50E370E0100D1
:107EC000637AC60D130EF00F6374CE0013038000A7
:107ED000335E6600B386C60103CE0600330E6E0025
:107EE000130300023303C341630C0300B395650021
:107EF000335EC501331866003367BE00B3176500F3
:107F0000135E0801B355C703131508011355050186
:107F100093D607013376C703B305B50213160601DE
:107F2000B366D60063FAB600B386060163E60601BF
:107F300063F4B600B3860601B386B64033F7C603D2
:107F40009397070193D70701B3D6C603B306D502AB
:107F500013150701B367F50063FAD700B38707016C
:107F600063E6070163F4D700B3870701B387D740FF
:107F700033D5670093050000638C0800B307A04069
:107F80003337F000B305B04013850700B385E540F3
:107F900067800000370E000113030001E36AC6F397
:107FA000130380016FF0DFF2631606001308100060
:107FB00033586802370701006372E80A1307F00FAD
:107FC000637407011303800033576800B386E6002B
:107FD00003C6060033066600130300023303C340E2
:107FE00063180308B385054193560801131508016A
:107FF0001355050113D6070133F7D502B3D5D502C2
:10800000131707013367C700B305B502637AB700DA
:1080100033070701636607016374B700330707017D
:10802000B305B74033F7D5029397070193D70701FC
:10803000B3D5D502B305B50213150701B367F50033
:1080400063FAB700B387070163E6070163F4B7007B
:10805000B3870701B387B7406FF09FF1370700017F
:1080600013030001E362E8F6130380016FF0DFF50C
:108070003318680033DEC500935E08013356C5002F
:10808000B31765003355DE03B39565003366B6005C
:108090009315080193D50501935606013377DE0346
:1080A0003385A502131707013367D700637AA7004A
:1080B00033070701636607016374A70033070701ED
:1080C000B306A74033F7D60313160601135606016D
:1080D000B3D6D60313170701B386D502B365C7001D
:1080E00063FAD500B385050163E6050163F4D500A5
:1080F000B3850501B385D5406FF01FEFE3EED5E6FC
:108100003708010063FC0605930EF00F33B8DE005C
:108110001318380033DE0601178301001303831997
:108120003303C301834E0300130E0002B38E0E010E
:10813000330EDE41631E0E0263E4B600636AC500BF
:10814000B307C540B385D5403335F5003387A54027
:1081500013850700930507006FF01FE23703000146
:1081600013080001E3E866FA130880016FF09FFA34
:108170003357D601B396C601B366D700B357D501BE
:1081800033D7D501B395C501B3E7B70093D5060141
:108190003373B702139F0601135F0F0113D8070152
:1081A0003316C6013315C5013357B7021313030144
:1081B00033680301B30FEF0213030700637EF80176
:1081C0003308D8001303F7FF6368D8006376F8011B
:1081D0001303E7FF3308D8003308F841B37FB80230
:1081E0003358B802939F0F01B3050F03139F070184
:1081F000135F0F0133EFEF0113070800637EBF0029
:10820000330FDF001307F8FF6368DF006376BF00FA
:108210001307E8FF330FDF0013130301B70F01004B
:108220003363E3009387FFFF13580601330FBF400A
:10823000B375F30013530301B377F6003387F502E8
:10824000B307F302B385050333030303B385F500D6
:10825000135807013308B8006374F8003303F301BF
:10826000B70701009387F7FF935508013378F800AB
:10827000131808013377F700B38565003307E8006A
:108280006366BF00631EBF00637CE5003306C74022
:108290003337C700B385D540B385E54013070600E3
:1082A0003307E5403335E500B305BF40B385A5404E
:1082B000B397D5013357C70133E5E700B3D5C501FF
:1082C0006FF09FCB93870500130806001387060005
:1082D000130305006396062897880100938888FD9C
:1082E00063F6C50E370701006378E60C1307F00F3D
:1082F0003337C70013173700B356E600B388D800EA
:1083000083C608003387E60093060002B386E64082
:10831000638C0600B397D7003357E5003318D600B7
:10832000B365F7003313D50013550801B3D7A50281
:1083300013160801135606019356030133F7A502DD
:10834000B305F60213170701B366D70013870700BA
:1083500063FEB600B38606011387F7FF63E80601E4
:1083600063F6B6001387E7FFB3860601B386B6400F
:10837000B3F7A6021313030113530301B3D6A602E6
:108380009397070133E36700B305D6021385060010
:10839000637CB300330368001385F6FF6366030153
:1083A0006374B3001385E6FF131707013367A70053
:1083B000930500006F00400EB7060001130700018F
:1083C000E36CD6F2130780016FF01FF3631606000B
:1083D0009306100033D8C602B70601006372D80CAA
:1083E0009306F00F63F4060113078000B356E8000C
:1083F000B388D80083C60800B386E60013070002DE
:108400003307D7406318070AB38707419305100065
:10841000135608019318080193D8080193560301D5
:1084200033F7C702B3D7C70213170701B366D700E4
:108430003385F8021387070063FEA600B3860601A2
:108440001387F7FF63E8060163F6A6001387E7FFCB
:10845000B3860601B386A640B3F7C6021313030121
:1084600013530301B3D6C6029397070133E36700A2
:10847000B388D80213850600637C130133036800B8
:108480001385F6FF63660301637413011385E6FF2A
:10849000131707013367A700130507006780000063
:1084A000B706000113070001E362D8F41307800147
:1084B0006FF0DFF33318E800B3D5D7003313E500CE
:1084C000B356D50013550801B397E70033F7A5025B
:1084D000B3E8F6009317080193D7070113D60801F4
:1084E000B3D5A502131707013367C700B386B702D8
:1084F00013860500637ED700330707011386F5FF57
:10850000636807016376D7001386E5FF3307070129
:10851000B306D74033F7A6029398080193D8080111
:10852000B3D6A60213170701B385D702B3671701A5
:108530001387060063FEB700B38707011387F6FFB2
:1085400063E8070163F6B7001387E6FFB387070107
:10855000B387B74093150601B3E5E5006FF05FEB15
:1085600063E6D5183707010063F4E6041308F00F3B
:108570003337D8001317370033D8E600978501004A
:10858000938545D3B385050103C805009305000213
:108590003308E800B3850541639605021307100010
:1085A000E3ECF6EE3335C500134715006FF0DFEE50
:1085B000B705000113070001E3E0B6FC13078001D3
:1085C0006FF09FFB33570601B396B600B366D70032
:1085D00093DE060133D70701B378D703B397B7000B
:1085E000335805013363F8009397060193D70701C9
:1085F000135803013316B6003357D7039398080175
:1086000033E80801338FE702130E0700637EE801A9
:108610003308D800130EF7FF6368D8006376E801CB
:10862000130EE7FF3308D8003308E841B378D803C6
:108630003358D80393980801B38E070393170301A7
:1086400093D70701B3E7F8001307080063FED701CB
:10865000B387D7001307F8FF63E8D70063F6D701A5
:108660001307E8FFB387D700131E0E01B387D74166
:10867000B70E01003367EE001388FEFF3373070166
:10868000935807013378060113560601330E03038E
:108690003388080393560E013303C30233030301E7
:1086A000B3866600B388C80263F40601B388D801B4
:1086B00013D60601B308160163E61703E39A17CF32
:1086C000B70701009387F7FFB3F6F600939606010C
:1086D000337EFE003315B500B386C6019305000056
:1086E000E37CD5DA1307F7FF6FF09FCC930500000A
:1086F000130700006FF05FDA930806001387060087
:108700009307050013880500639C062297860100E5
:10871000938646BA63FCC50C37030100637E660A84
:108720001303F00F6374C300130780003353E60094
:10873000B386660003CE060013030002330EEE007C
:108740003303C341630C0300B3956500335EC50179
:10875000B31866003368BE00B317650013D608016E
:108760003377C802139508011355050193D6070105
:108770003358C80213170701B366D700330805033F
:1087800063FA0601B386160163E6160163F4060177
:10879000B3861601B386064133F7C60293970701E5
:1087A00093D70701B3D6C602B306D5021315070146
:1087B000B367F50063FAD700B387170163E61701C3
:1087C00063F4D700B3871701B387D74033D5670069
:1087D00093050000678000003703000113070001C4
:1087E000E36666F4130780016FF05FF4631606001A
:1087F00013061000B35816033706010063F2C80AC7
:108800001306F00F637416011307800033D6E800D7
:10881000B386C60003CE060013030002330EEE003B
:108820003303C34163180308B385154113D7080107
:10883000139508011355050113D60701B3F6E50298
:10884000B3D5E50293960601B3E6C600B305B502BB
:1088500063FAB600B386160163E6160163F4B60048
:10886000B3861601B385B640B3F6E50293970701C8
:1088700093D70701B3D5E502B305B50213950601F9
:10888000B367F50063FAB700B387170163E6170112
:1088900063F4B700B3871701B387B7406FF01FF3D6
:1088A0003706000113070001E3E2C8F61307800151
:1088B0006FF0DFF5B398680033D7C501B3176500D3
:1088C000335EC50113D50801B376A702B3956500E1
:1088D000336EBE009395080193D5050113560E0122
:1088E0003357A70293960601B3E6C6003387E50225
:1088F00063FAE600B386160163E6160163F4E60048
:10890000B38616013386E640B376A602131E0E0127
:10891000135E0E013356A602939606013386C502F6
:10892000B3E5C60163FAC500B385150163E6150119
:1089300063F4C500B3851501B385C5406FF01FEF23
:10894000E3EAD5E83707010063FCE604930EF00F75
:1089500033B7DE001317370033D3E60097880100E2
:1089600093884895B388680083CE0800130E0002F0
:10897000B38EEE00330EDE41631E0E0263E4B600DA
:10898000636AC500B307C540B385D5403335F500EC
:108990003388A54013850700930508006FF09FE317
:1089A000B708000113070001E3E816FB1307800175
:1089B0006FF09FFA3357D601B396C601B366D7005E
:1089C000B357D50133D7D501B395C501B3E7B70088
:1089D00093D506013373B702139F0601135F0F018E
:1089E00093D807013316C6013315C5013357B702B3
:1089F00013130301B36813013308EF0213030700D5
:108A000063FE0801B388D8001303F7FF63E8D800BA
:108A100063F608011303E7FFB388D800B388084161
:108A2000B3FFB802B3D8B802939F0F01B3051F0379
:108A3000139F0701135F0F0133EFEF011387080046
:108A4000637EBF00330FDF001387F8FF6368DF002A
:108A50006376BF001387E8FF330FDF0013130301B2
:108A6000B70801003363E3009387F8FF135806014A
:108A7000330FBF40B375F30013530301B377F60010
:108A80003387F502B307F302B3850503330303030A
:108A9000B385F500135807013308B8006374F80074
:108AA00033031301B70701009387F7FF93550801BC
:108AB0003378F800131808013377F700B3856500A1
:108AC0003307E8006366BF00631EBF00637CE500F8
:108AD0003306C7403337C700B385D540B385E5407B
:108AE000130706003307E5403335E500B305BF4003
:108AF000B385A540B397D5013357C70133E5E700E8
:108B0000B3D5C5016FF01FCD978701009387879973
:108B100083A607001787010013078797032707001D
:108B200023A2A600637EE5001787010013070797BD
:108B30000325070083A50700938545006F709FC438
:108B4000130101FF23248100232611001787010050
:108B500013070795130405000325070083A50700E5
:108B600093854500EF701FC2978701009387879018
:108B700083A707006376F4009787010023AC878EF4
:108B80008320C100032481001301010167800000DC
:108B9000978701009387079103A7070083A6070023
:108BA000832747049387F7FF2322F70483A746040C
:108BB000639407007360043067800000130101FEB6
:108BC000232C8100232A91001304050093840500BF
:108BD000232821012326310123244101232251018D
:108BE000232E1100EFA0CFBE832704000329040128
:108BF000B7090001B3E59700930AC4002320B4002D
:108C0000930400009389F9FF370A00020327040048
:108C100063822A050326090013050900B36547018D
:108C2000B37636019317560033F7E600032949005F
:108C300063C60700631607006FF05FFDE398E6FC6C
:108C40009317760063D40700B3E4D400EFB08FFF2E
:108C50006FF0DFFB93C4F4FFB3F4E400232094002F
:108C6000EFA08FEA032504008320C10103248101C2
:108C700083244101032901018329C100032A8100C2
:108C8000832A41001301010267800000130101FFE4
:108C90002326110023248100EFE09F8417E7FFFFC4
:108CA0001307C773930600001306100093054006D0
:108CB0001775010013050575EFC01FAF63020502AC
:108CC00013040500EFA04FB21306050013070000C0
:108CD000930600009305100013050400EFC0DFBEEB
:108CE000EF905FFC8320C100032481001305000086
:088CF00013010101678000007F
:02000004800278
:10000000C467FEFF3469FEFFD067FEFF3469FEFF60
:100010003469FEFF3469FEFF3469FEFFF867FEFFB6
:100020003469FEFF3469FEFF2068FEFF3068FEFF82
:100030003469FEFF4868FEFF5868FEFF5868FEFFFF
:100040005868FEFF5868FEFF5868FEFF5868FEFFBC
:100050005868FEFF5868FEFF5868FEFF3469FEFFCF
:100060003469FEFF3469FEFF3469FEFF3469FEFF28
:100070003469FEFF3469FEFF3469FEFF3469FEFF18
:100080003469FEFF3469FEFF3469FEFF3469FEFF08
:100090003469FEFF3469FEFF3469FEFF3469FEFFF8
:1000A0003469FEFF3469FEFF3469FEFF3469FEFFE8
:1000B0003469FEFF3469FEFF3469FEFF3469FEFFD8
:1000C0003469FEFF3469FEFF3469FEFF3469FEFFC8
:1000D0003469FEFF3469FEFF3469FEFF3469FEFFB8
:1000E0003469FEFF3469FEFF3469FEFF3469FEFFA8
:1000F0003469FEFF3469FEFF3469FEFF3469FEFF98
:100100009C68FEFFC468FEFF3469FEFF3469FEFF91
:100110003469FEFF3469FEFF3469FEFF3469FEFF77
:100120003469FEFF2469FEFF3469FEFF3469FEFF77
:10013000D465FEFFDC66FEFF3469FEFF3469FEFF16
:100140002C67FEFF3469FEFFA467FEFF3469FEFFE3
:100150003469FEFFEC67FEFF906DFEFFFC6DFEFF55
:100160009C6DFEFFFC6DFEFFFC6DFEFFFC6DFEFF57
:10017000FC6DFEFF346CFEFFFC6DFEFFFC6DFEFFB0
:100180005C6CFEFF6C6CFEFFFC6DFEFF846CFEFF82
:10019000946CFEFF946CFEFF946CFEFF946CFEFF6B
:1001A000946CFEFF946CFEFF946CFEFF946CFEFF5B
:1001B000946CFEFFFC6DFEFFFC6DFEFFFC6DFEFF10
:1001C000FC6DFEFFFC6DFEFFFC6DFEFFFC6DFEFF97
:1001D000FC6DFEFFFC6DFEFFFC6DFEFFFC6DFEFF87
:1001E000FC6DFEFFFC6DFEFFFC6DFEFFFC6DFEFF77
:1001F000FC6DFEFFFC6DFEFFFC6DFEFFFC6DFEFF67
:10020000FC6DFEFFFC6DFEFFFC6DFEFFFC6DFEFF56
:10021000FC6DFEFFFC6DFEFFFC6DFEFFFC6DFEFF46
:10022000FC6DFEFFFC6DFEFFFC6DFEFFFC6DFEFF36
:10023000FC6DFEFFFC6DFEFFFC6DFEFFFC6DFEFF26
:10024000FC6DFEFFFC6DFEFFFC6DFEFFFC6DFEFF16
:10025000FC6DFEFFFC6DFEFFD86CFEFF146DFEFF13
:10026000FC6DFEFFFC6DFEFFFC6DFEFFFC6DFEFFF6
:10027000FC6DFEFFFC6DFEFFFC6DFEFF806DFEFF62
:10028000FC6DFEFFFC6DFEFF086AFEFF5C6BFEFF6F
:10029000FC6DFEFFFC6DFEFFEC6BFEFFFC6DFEFFD8
:1002A000186CFEFFFC6DFEFFFC6DFEFFF06DFEFFA7
:1002B000000102020303030304040404040404040D
:1002C00005050505050505050505050505050505DE
:1002D00006060606060606060606060606060606BE
:1002E00006060606060606060606060606060606AE
:1002F000070707070707070707070707070707078E
:10030000070707070707070707070707070707077D
:10031000070707070707070707070707070707076D
:10032000070707070707070707070707070707075D
:10033000080808080808080808080808080808083D
:10034000080808080808080808080808080808082D
:10035000080808080808080808080808080808081D
:10036000080808080808080808080808080808080D
:1003700008080808080808080808080808080808FD
:1003800008080808080808080808080808080808ED
:1003900008080808080808080808080808080808DD
:1003A00008080808080808080808080808080808CD
:1003B000546D725100000000546D7220537663003A
:1003C000286E756C6C2900004572726F7220696E20
:1003D00020787878207461736B73200D0A00000018
:1003E0006D69616F750A00006D69616F75320A0091
:1003F00068756E6772790A0054696D657232000023
:10040000436865636B54696D65720000536574548D
:0C04100078000000536574527800000072
:10041C001000000000000000017A5200017C010174
:10042C001B0D02001000000018000000347AFEFFC3
:10043C005804000000000000100000002C00000018
:10044C00787EFEFF34040000000000001000000065
:10045C00400000009882FEFF100400000000000025
:10050000FC8F010009000000FFFF0000FFFF00005A
:0405100001000000E6
:040000058000004037
:00000001FF
